:1080000000000120E51D01003DF500003DF50000E8
:108010003DF500003DF500003DF5000000000000CA
:108020000000000000000000000000003DF500001E
:108030003DF50000000000003DF500001D86000039
:108040003DF500003DF500003DF500003DF5000068
:108050003DF500003DF500003DF500003DF5000058
:108060003DF500003DF500003DF500003DF5000048
:108070003DF500003DF500003DF500003DF5000038
:108080003DF500003DF500003DF500003DF5000028
:108090003DF500003DF500003DF500003DF5000018
:1080A0003DF50000D5E500003DF500003DF5000080
:1080B0003DF500003DF500003DF500003DF50000F8
:1080C0003DF500003DF500003DF500003DF50000E8
:1080D0003DF500003DF500003DF50000E9E1000040
:1080E0003DF500003DF500003DF500003DF50000C8
:1080F0003DF500003DF500003DF500003DF50000B8
:108100003DF500003DF500003DF500003DF50000A7
:108110003DF50000590701003DF500003DF5000068
:108120003DF500003DF500003DF500003DF5000087
:108130003DF500003DF500003DF500003DF5000077
:108140003DF500003DF50000718700003DF50000A1
:108150003DF500003DF500003DF500003DF5000057
:108160003DF5000025E200003DF500003DF5000072
:108170003DF500003DF500003DF500003DF5000037
:088180003DF500003DF5000093
:10840000FFFFFFFFFFFFFFFFFFFFFFFF7EF9FFFF03
:1084100010B5054C237833B9044B13B10448AFF3BE
:1084200000800123237010BD0086FF1F00000000A4
:10843000442301000C4B43B10C480D4910B5AFF378
:1084400000800C48036823B910BD0A48036833B99B
:108450007047094B002BF7D0BDE810401847064B7A
:10846000002BF5D0184700BF000000004423010096
:108470000486FF1F7485FF1F0000000080F3118831
:1084800070472F4B41F238015A5842F478525A50F3
:108490002C4A927902F00C020C2A4FD041F244028D
:1084A0002949995003F558339A78110748BF9A78AB
:1084B000264944BF42F008029A70214B41F244021F
:1084C000995041F204015A5842F4803242F0C002FD
:1084D0005A501A6842F440221A6003F5E833242205
:1084E0005A701B4A80211170A2221A70DA7802F0A9
:1084F0001F02DA7003221A7100225A719A799207C8
:10850000FCD59A79D006FCD40E4B19469A7902F024
:108510000C02082AFAD140225A718B7903F00C031D
:10852000082BFAD1074B1A4699794906FCD5222126
:108530001970937903F00C030C2BFAD1704700BF2C
:1085400000700440004006400000330100001301A9
:10855000005006402B4B5A7902F0E0025A711A790A
:1085600002F0F8021A71284A136843F004031360FA
:10857000264A136823F0784323F001031360244B49
:108580001A7802F08C0242F050021A705A7802F007
:108590009C0242F040025A709A7802F0E6029A7009
:1085A0001C4A0023137083F311881B4B012283F8AC
:1085B000182383F81923022283F83C2383F83D23F0
:1085C00083F84B2383F84C2383F84D2383F84E2301
:1085D00083F84F23032283F81F2383F8212383F892
:1085E000232383F8252383F84223042283F82723B7
:1085F000052283F84923062283F83B23072283F8C8
:108600003523704700F007404080044000D0004010
:1086100000D0074000E0074000E100E00C4A13688A
:10862000013313600B4A1368013313600A4B1A6855
:108630003AB11A68013A1A601B6813B9074B012254
:108640001A70074B1A6812B11A68013A1A6070471B
:108650001C86FF1F90070020200300201C03002021
:1086600024030020024B034A5A6007221A60704715
:1086700010E000E000770100014B1868704700BF70
:108680001C86FF1F1449154B41F22802072888BF9A
:10869000002010B553F82030114CB4FBF3F48B5884
:1086A00043F480638B500F4B4FF440729A63422027
:1086B000DA6306F061FF0C4B0022DA709A709A714F
:1086C000DA725A71C4F30422E4B21A705C70DA7878
:1086D00042F02C02DA7010BD0070044090200100BE
:1086E000C0C62D0000B0044000A00E40094A136827
:1086F00051680133202B08BF00238B4208D011683A
:10870000114408721360044AD37843F08003D37095
:10871000704700BF2086FF1F00A00E400A4B996AD9
:10872000DA6A91420DD09A6A511C1A44996292F801
:10873000302002709A6A202A01D100229A62012018
:1087400070470020704700BF2086FF1F044B1A7837
:1087500002F0FF0012B100221A700120704700BF22
:108760001C030020014B1865704700BF2086FF1FC7
:1087700030B526480179C9B28C0617D5244BDA6A80
:108780009C6A0132202A08BF0022A2421BBFDC6A79
:10879000C579C27918191EBFEDB280F83050DA627F
:1087A0001C4A052010601A6D1B4B1A604A0608D53A
:1087B0001A4B4FF480529A60144AD37803F0BF03E7
:1087C000D3700B061BD5144B1868C0B9104B196831
:1087D0005A68914214D0114A4FF4805151605A683E
:1087E000511C1A445960117A084AC9B2D1715968AA
:1087F000202908BF5860D37843F04003D37030BDC0
:10880000024AD37803F07F03F8E700BF00A00E40D0
:108810002086FF1F200300202403002080F00F404B
:1088200062B67047FFF7FCBF72B67047FFF7FCBF38
:108830004FF0E02318B1034AC3F80C2D7047024AE9
:10884000FAE700BF0400FA050100FA05F7B5464C47
:108850004649474D474E4FF4807306226360A3603C
:1088600023618A6010224A601E224A61424A536292
:108870009364D3644FF400226A61AA603F4A4FF4C4
:10888000907050621363936402F5342280324FF487
:10889000905090604FF48020506000F590505061EF
:1088A000374A40F20310106050609060D060106151
:1088B00050619061D06133480022426132480361C7
:1088C00043618361836600F5322000F58070866025
:1088D0004661082623601046E360B4460A242B460E
:1088E00017468E46C1F804C00197019DB5F57A7F01
:1088F00030D3DEF810508E60ED0748BF013001978D
:10890000019DB5F57A7F29D3DEF81050ED0758BFE9
:108910000132013CE6D10A281C4923D10A2A21D17F
:1089200001220A70104A4FF4E0611160D16002F533
:108930003622102191604FF400225A600E4A4FF403
:108940008071116001225A605A6942F001025A6135
:1089500003B0F0BD019D01350195C6E7019D0135CC
:108960000195CDE70022DCE70090044000F00F40C5
:1089700040F00F407000000400A0044000B004402C
:1089800000C00440C0F00F4000D004407403002039
:10899000F7B5104B1B78D3B10F4B104D02210F468A
:1089A000042000241E465F6098600194019AAA4248
:1089B00009D9B16070600194019AAA42F3D8019A72
:1089C00001320192F8E7019A01320192EEE703B019
:1089D000F0BD00BF7403002000F00F401FA107008E
:1089E000032806D8DFE800F00206080A1022054B2B
:1089F0005A6070472022FAE74022F8E74FF0806281
:108A0000F5E700BF00F10F40032806D8DFE800F0CB
:108A10000206080A1022054B9A6070472022FAE7E6
:108A20004022F8E74FF08062F5E700BF00F10F4009
:108A300010B50021044644FA01F3DB07C8B205D59E
:108A4000FFF7CEFF01310829F5D110BDFFF7DCFF9C
:108A5000F8E708B5032813D8DFE800F0020C0E1081
:108A6000002005F045FC43F27C03984294BF0020AF
:108A7000012008BD0120F4E70220F2E70320F0E71F
:108A8000002008BD032817D8DFE800F002070C110A
:108A90000A4B1868C0F300107047084B1868C0F301
:108AA00040107047054B1868C0F380107047034BA7
:108AB0001868C0F3806070470020704700F10F40D5
:108AC00070B5002425460126E0B2FFF7C2FF18B1B9
:108AD00006FA04F31D43EDB20134082CF4D1284604
:108AE00070BD024B1869C043C0B27047C0F00F4060
:108AF00037B50446FFF7C0FD0546FFF7BDFD401B37
:108B00000028B8BF40420128F7DD0020012C8DF875
:108B100004008DF8050010D007D3022C11D00306F5
:108B200048BF60F0FF0003B030BD022201A99020D1
:108B300005F00CFE9DF80400F1E7022201A9922045
:108B4000F6E7224601A99420F2E708B5082005F0CF
:108B5000CFFB5E2811D9134B1A780AB901221A707B
:108B6000082005F0C5FBA9280FD90F4B1B7863B966
:108B70000E4B4FF400725A6008BD082005F0B8FB98
:108B80005428EDD80022074BE9E7082005F0B0FB98
:108B9000952802D9044B1B781BB1044B4FF400728B
:108BA0009A6008BD7486FF1F4F03002080F00F40BD
:108BB000034B1878013801288CBF00200120704732
:108BC0007486FF1F034B1878012806BF02221A7013
:108BD000002070477486FF1FC0B206F09DBAC0B275
:108BE00006F088BA08B508F0DBFB06F099FE06F03F
:108BF00049FEBDE8084008F055BC38B5054606F00A
:108C000097FD08280AD900242819013406F010FE1F
:108C1000092CF9D106F040FE012038BD002038BDF6
:108C2000092106F0A5BD002007F032B822492348EB
:108C300041F23C028B5843F440538B50204B0121AE
:108C400019601A6802431A601E4ADA601A61DA6A09
:108C500042F08052DA621A6822F001021A601A6841
:108C600022F000621A60184A4FF4007313605360D8
:108C70009360D360136153619361D361A2F5F032C5
:108C800011601168014311601049D16001F52001A4
:108C90001161D16A41F08051D162116821F0010166
:108CA0001160116821F00061116002F5E8329362F1
:108CB000D36213645364704700700440000C1F803B
:108CC00000C002400300013E00B004400400513ED9
:108CD000FF2810B54FEA004323D82B4C03F47C1334
:108CE0008AB141F000610B436363E36A002BFCDA55
:108CF000254BDA6AD000FCD5986BDA6A42F0104254
:108D0000C0B2DA6210BD41F000410B436363E36A15
:108D1000002BFCDAA06BE36A43F01043C0B2E362BD
:108D200010BDB0F5007F17D2184C03F47C135AB174
:108D300041F000610B436363E36A002BFCDA134BE1
:108D4000DA6AD100FCD5D7E741F000410B436363F9
:108D5000E36A002BFCDADDE70D4C03F47C135AB117
:108D600041F000610B436363E36A002BFCDA084BBC
:108D7000DA6AD200FCD5BFE741F000410B436363E0
:108D8000E36A002BFCDAC5E700C0024000D00240D5
:108D900000C00A4010B5FFF76FFC0446FFF76CFCFB
:108DA000001B0028B8BF40420628F7DD10BD07B5FC
:108DB000030A8DF805008DF80610032201A9A020F2
:108DC0008DF8043005F09CFCFFF7E4FF03B05DF87C
:108DD00004FBF0B5154600228BB00F461446AC429A
:108DE00001D10BB0F0BD0AAB1344395D03F8221C6E
:108DF000531CC618F10602D0691E8C420DD1030A1D
:108E00008DF80500033201A9A0208DF8043005F08B
:108E100077FCFFF7BFFF3046002301341A46DEE738
:108E20001FB5030A8DF80C30022203AB8DF80D003C
:108E300000921946A02005F0AFFC9DF80C0005B08B
:108E40005DF804FB1FB5030A8DF80C308DF80D009A
:108E500000920B46022203A9A02005F09DFC05B05C
:108E60005DF804FB30B4C0EBC000074C0D68255022
:108E700022188C8894808B79937100F5B04007227A
:108E800030BCFFF7A6BF00BF7586FF1F054BC0EBC8
:108E9000C000184403680B6083888B8083798B71D2
:108EA000704700BF7586FF1F30B500238BB001AD42
:108EB0001A465A550133222BFBD14FF4B044230AF2
:108EC0008DF8054022222946A02020348DF8043058
:108ED00005F016FCFFF75EFFB4F5484FEFD10B49E4
:108EE00000220C461346C2EBC20020440132B2F508
:108EF000805F0B704B708B70C37003714371837113
:108F000001F10701EFD10BB030BD00BF7586FF1F27
:108F100013B50C46C0EBC0000722694600F5B0400F
:108F2000FFF790FF9DF8002023789A4212D19DF818
:108F3000012063789A420DD19DF80220A3789A42CD
:108F400008D1DDF80300D4F80330C31A5842584161
:108F500002B010BD0020FBE77047F0B545F2FF708E
:108F600085B0FFF75DFF552803D13C4B1B78002BE4
:108F700043D0002145F2FF70FFF719FFFFF794FF80
:108F800040223749374F384E0020FFF722FF4FF479
:108F9000B7654024204640223946FFF71AFF403487
:108FA000284660223146FFF714FFB4F5807F05F1B3
:108FB0006005EFD104AD002345F8043D4FF4D364C0
:108FC00040F678062046042229460434FFF701FFC4
:108FD000B442F7D1002303934FF4FF6440F6D80660
:108FE0002046042229460434FFF7F3FEB442F7D1A9
:108FF000552145F2FF70FFF7DAFE402218491B4D5C
:10900000194E0020FFF71EFF402210461849FFF7B7
:1090100019FF402217498020FFF714FF402216490C
:10902000C020FFF70FFF002428196022314660346A
:1090300008F04CFAB4F5907FF6D158238DF808303B
:1090400000238DF809304FF4E043009302220B4BCC
:1090500002A9A02005F0A0FB05B0F0BD740300201C
:109060000C80FF1F20210100C0200100C804002047
:1090700098030020FC030020600400207586FF1F79
:10908000044B9B78022B044B8CBF042203221A70E2
:10909000704700BF780600209407002038B5014CC7
:1090A000637801E078060020FF2B00F23F85DFE8BF
:1090B00013F0010217022C024B02570262026B02EC
:1090C00074027D0286028C0295029E02B202C602E2
:1090D000CF02DA02E302EC02F70200030B031403EF
:1090E0001B0322032903300337033E0352033D05CC
:1090F0003D053D055B0362033D053D053D053D0521
:109100003D053D053D053D053D053D053D053D054F
:109110003D053D053D0569033D053D053D053D0515
:109120003D053D053D053D053D053D053D053D052F
:109130003D053D053D053D053D053D053D053D051F
:109140003D053D053D053D053D053D053D053D050F
:109150003D053D053D053D053D053D053D053D05FF
:109160003D053D053D053D053D053D053D053D05EF
:109170003D053D053D053D053D053D053D053D05DF
:109180003D053D053D053D053D056F037803810324
:1091900093039C03A503AE03B703C003C903D20323
:1091A000DB03E403ED033D05F603FD0306040F04B2
:1091B00018041F0426043D052E0435043C04420413
:1091C0003D054B0455045F043D0568043D053D0520
:1091D0003D053D053D053D053D053D053D053D057F
:1091E0003D053D053D053D053D053D053D053D056F
:1091F0003D053D053D05000115011B012101310122
:10920000410147014D01530159015F0165016B01A6
:109210003D053D0571013D053D0577017D018A0153
:109220003D05A701AD01B301D001D601DC01E30189
:10923000EF01F50173047C04880495049C043D054A
:109240003D05A304AC04B2043D05FB013D05BB0490
:10925000D104E504EB04F7043D0500050A051405F7
:109260003D053D053D053D053D053D053D053D05EE
:109270003D053D053D053D053D053D053D053D05DE
:109280003D053D053D053D053D053D053D053D05CE
:109290003D053D053D053D053D053D053D053D05BE
:1092A0003D053D051E053D0529053D053D053D05E1
:1092B0003305A07805F021FD994B5860994B1B7838
:1092C0005BB1974B5A68984B1A60984B002A40F054
:1092D00032841A6842F008021A6038BDA07805F09E
:1092E00036FD8F4B5860E9E7A07805F03EFD8C4BCA
:1092F0005860E3E7A0788A4D05F029FDA37820B9EE
:10930000184605F04CFD6860D8E7184605F034FDB6
:109310006860D3E7A078824D05F019FDA37820B9E5
:10932000184605F0E3FC6860C8E7184605F030FD14
:109330006860C3E7A07805F0C7FC794B5860BDE7CB
:10934000A07805F0D0FD764B5860B7E7A07805F01F
:10935000AAFD734B5860B1E7A07805F0ABFD704BE8
:109360005860ABE7A07805F097FD6D4B5860A5E716
:10937000A07805F0A6FD6A4B58609FE7A07805F03D
:10938000B9FD674B586099E7A07805F0A1FD644BE3
:10939000586093E7A07805F0C5FC614B58608DE7F5
:1093A000A378634AD25C5E4B5A6087E7A278614932
:1093B000642303FB02136049186951F82220904787
:1093C000574B58607AE71421A078554D05F03CFBC7
:1093D0000028D5BF6FF07F43584B6B6093FBF0F0D4
:1093E000544AA378C8BF6860642101FB03231B7E35
:1093F000002B7FF463AF686806F097F868605DE75C
:10940000A07805F0ABFC464B586057E7A07805F014
:109410007BFC434B586051E71321A078404D05F089
:1094200013FB0028D5BF6FF07F43444B6B6093FB69
:10943000F0F0404AA378C8BF6860642101FB0323B1
:109440001B7E002B7FF43AAF686806F06EF8686008
:1094500034E7A07805F0D9FD314B58602EE7A078AD
:1094600005F0DAFD2E4B586028E77121A07805F051
:10947000EBFA2B4B586021E70021A07805F0E4FAC5
:1094800010F0040F264B14BF012200225A6015E78A
:10949000A07805F0B3FD224B58600FE7A07805F0E7
:1094A000A6FD1F4B586009E7A07805F092FD1C4B04
:1094B000586003E7A0781A4D03F072FDA3783721B6
:1094C00020B9184605F088FE6860F7E6184605F0F2
:1094D00083FEA2781A4B53F82230C01A6860EDE67A
:1094E000A078184A0E4D602343432121D35C1BB959
:1094F00005F072FE6860E1E605F06EFEA278104BA2
:1095000053F82230C01A6860D8E60B4BA0782421AB
:1095100053F8204005F060FEA047014B5860CDE6AF
:10952000940700208F07002080070020800600207D
:109530004C0300209803002078F6FF1F0024F4005D
:1095400040030020C80400209F4BA078222153F83C
:10955000204005F041FE0002A0479C4B5860ADE65C
:10956000A278994B03EB820153F82230C8689847E0
:10957000964B5860A2E6964AA378642101FB032328
:109580009A6A924B5A6099E6914AA378642101FB4A
:1095900003235A7A8D4B5A6090E68D4AA378642152
:1095A00001FB03239A7A894B5A6087E60F21A07842
:1095B00005F012FE854B00F0010058607EE6A078B1
:1095C00005F0ACFF814B586078E60F21A07805F0DC
:1095D00003FE7E4BC0F3002058606FE60F21A07899
:1095E00005F0FAFD794BC0F3C010586066E6012122
:1095F000A07805F0F1FD830741BF744A536843F03A
:109600000103536005077FF559AE704A536843F074
:109610000203536052E60121A07805F0DDFDC40786
:1096200041BF6A4A536843F00103536041077FF525
:1096300045AE664A536843F0020353603EE6644A0F
:10964000A378642101FB0323DA7D604B5A6035E681
:109650005D4BA078252153F8204005F0BDFDA047C3
:109660005A4B58602AE65A4AA378642101FB032327
:109670001A6B564B5A6021E6554AA378642101FBC8
:109680000323DA6A514B5A6018E64F4BA078272122
:1096900053F8204005F0A0FDA0474C4B58600DE664
:1096A0004B4AA378642101FB03235A6B474B5A6052
:1096B00004E6454BA078262153F8204005F08CFDA8
:1096C000A047424B5860F9E5414AA378642101FB69
:1096D00003239A6B3D4B5A60F0E52D21A07805F0ED
:1096E0007BFD3A4B5860E9E52E21A07805F074FD2A
:1096F000364B5860E2E52F21A07805F06DFD334B25
:109700005860DBE53021A07805F066FD2F4B5860EE
:10971000D4E53321A07805F05FFD2C4B5860CDE5F2
:109720003421A07805F058FD284B5860C6E501218A
:10973000A07805F051FD420641BF244A536843F02A
:109740000103536003067FF5B9AD204A536843F027
:1097500002035360B2E50121A07805F03DFD1B4BEB
:10976000C0F301205860A9E50121A07805F034FD7F
:1097700010F0100F86E60121A07805F02DFD10F005
:10978000200F7FE6A07804F027F8104B586095E58D
:10979000104AA378602101FB03235A680B4B5A60DF
:1097A0008CE50C4AA378602101FB03239A68074BE0
:1097B0005A6083E5074AA378602101FB03231A7BE3
:1097C000024B5A607AE500BF78F6FF1F940700202D
:1097D00098030020C8040020974AA378602101FB69
:1097E0000323DA89954B5A6068E5934AA378602190
:1097F00001FB03231A69914B5A605FE58E4AA378F7
:10980000602101FB03231A7D8C4B5A6056E58A4A7E
:10981000A378602101FB03235A7D884B5A604DE5F4
:10982000854AA378602101FB03231A6A834B5A609F
:1098300044E5814AA378602101FB03235A6A7F4BE8
:109840005A603BE57C4AA378602101FB03239A6AB6
:109850007A4B5A6032E5784AA378602101FB0323F2
:10986000DA6A764B5A6029E5734AA378602101FBD6
:1098700003231A6B714B5A6020E56F4AA37860216D
:1098800001FB03239A696D4B5A6017E56A4AA37876
:10989000602101FB0323DA69684B5A600EE57C21E5
:1098A000A07805F099FC654B586007E5624AA378FB
:1098B000602101FB03235A6B604B5A60FEE45E4A51
:1098C000A378602101FB03239A6B5C4B5A60F5E49B
:1098D000594AA378602101FB03239A7D574B5A60B4
:1098E000ECE4A278564B13441A7E544B5A60E5E4DC
:1098F0002021A07805F070FC504B5860DEE4A2787F
:10990000602353434C4AD25C4C4B5A60D6E46621E8
:10991000A07805F061FC494B5860CFE46521A07840
:1099200005F05AFC454B5860C8E4A07803F038FBBA
:10993000424B5860C2E4404AA378602101FB0323F4
:10994000DA6B3E4B5A60B9E43B4AA378602101FBD5
:10995000032393F84020394B5A60AFE4364AA3788A
:10996000602101FB032393F84120344B5A60A5E4A6
:10997000314AA378602101FB03235A6C2F4B5A60B4
:109980009CE40A21A07805F027FC2C4B00F00F0086
:10999000C0F10800586091E42A4AA378642101FBD1
:1099A00003231A7A254B5A6088E4A2782449642359
:1099B000534351F822202349C85890471F4B586001
:1099C0007CE4A2781F49642303FB02131C495868F6
:1099D00051F822209047194B58606FE41A4BA27837
:1099E00053F82220154B5A6068E4184BA27853F8BC
:1099F0002220124B5A6061E4124AA378642101FBD1
:109A000003239A7D0D4B5A6058E4A07804F078FF48
:109A10000A4B586052E40B4AA378642101FB0323EC
:109A20009A8F064B5A6049E4094BA27853F82220DA
:109A3000024B5A6042E400BFC80400209407002093
:109A400078F6FF1F980300202C030020E805002073
:109A500068030020A2783A493A4B8C5C0020586099
:109A60000CB101245C6088543749885C18B158688F
:109A700040F00200586000238B541FE4A378334A5F
:109A8000D25C304B5A6019E45021A07805F0A4FB59
:109A9000A2782F4B53F82230C01A2A4B58600DE49D
:109AA0002C4AA378642101FB0323DA69254B5A6011
:109AB00004E4284AA378642101FB03231A6A214B9A
:109AC0005A60FFF7FBBB234AA378642101FB032301
:109AD0005A6A1C4B5A60FFF7F1BB1E4AA3786421F7
:109AE00001FB03239A8A174B5A60FFF7E7BB194A19
:109AF000A378642101FB032393F83E20114B5A60A5
:109B0000FFF7DCBB0021A07805F066FB0D4BC0F32E
:109B100000705860FFF7D2BB0E4AA378642101FBA6
:109B200003231A7E074B5A60FFF7C8BB054B03227D
:109B30001A70FFF7C3BB1A6822F00802FFF7CCBB0C
:109B4000900300209407002050030020930300207E
:109B5000580300209803002038B5BE4A90780228A8
:109B6000144600F0EE80032800F0F280002840F058
:109B7000CC8153784D2B00F0A1803AD8452B79D079
:109B800016D8412B6DD004D8402B63D00322B24BA2
:109B90005EE0422B69D0442BF8D1B049D2F80330B3
:109BA00041F81C3F04221C20BDE83840FFF711B9E2
:109BB000492B6CD014D8462B61D0472BE6D1A74D4A
:109BC000D2F803302946042241F8083F0820FFF765
:109BD00000F92A8A29896879BDE8384004F0B8BBC1
:109BE0004B2B60D04C2BD1D19C4BD178997002205B
:109BF00033E0542B00F0838018D8512B6AD008D85A
:109C00004F2B60D0502BC1D1944BD1789975162031
:109C100023E0522B6BD0532BB8D1904DD2F80330A8
:109C20002946042241F8103F1020D0E7842B7ED033
:109C300008D8552B6FD0832BA8D1894BD2F803209D
:109C4000DA6138BD852B77D0FF2B9FD1D278854B39
:109C50001A7038BDD17845F2FF70BDE83840FFF783
:109C6000A6B87E4BD1781970F7E77C4BD178597044
:109C70000120F2E7794BD17859710520EDE777495A
:109C8000D2F8033041F80C3F04220C208CE7D27844
:109C9000724B1AB9DA75D97D1720DEE76E490122B9
:109CA000DA754A60F7E76D4CD178E1700320FFF771
:109CB0007EF8E078BDE83840FEF754BD674BD178B8
:109CC00059751520C9E7D2F80310644BC9B259760B
:109CD0001920C2E7614D2A7DD20704D5E378DB075E
:109CE00001D4FFF7E1F8E17829751420B5E75B4965
:109CF000D2F8033041F8203F0422202054E7D2F864
:109D00000330012B00F201815449D37801F81A3F46
:109D100001221A2048E7D2F80330012B00F2F58027
:109D20004E49D37801F81B3F01221B203CE74E4BE4
:109D3000D2F803201A6038BDD2F80320484B1A62CB
:109D400038BD5178494BD2F8032043F8212038BD63
:109D500053782E2B3FF61AAF01A252F823F000BF22
:109D60001D9E00002F9E0000419E00008D9B000064
:109D70008D9B00008D9B00008D9B00008D9B000043
:109D80008D9B0000539C0000539C0000539C0000DE
:109D90008D9B00008D9B00008D9B00008D9B000023
:109DA0008D9B00008D9B00008D9B00008D9B000013
:109DB0008D9B00008D9B00008D9B00008D9B000003
:109DC0008D9B00008D9B00008D9B0000759E000008
:109DD000819E00008D9E0000999E0000A59E0000BF
:109DE000B19E00008D9B00008D9B00008D9B0000AC
:109DF0008D9B00008D9B00008D9B0000BD9E000090
:109E0000C59E0000CF9E0000D99E0000E39E00008A
:109E1000ED9E0000F79E0000019F0000144BD4F857
:109E200003201A60FEF728FC0D4B586238BD104B1A
:109E3000D4F803205A60FEF71FFC094B986238BD26
:109E40000B4BD4F803209A60FEF716FC044BD86243
:109E500038BD00BF78060020940700200C80FF1F4B
:109E600078F6FF1F8E07002090070020A007002033
:109E7000F4050020D4F80330254ADBB2137638BD50
:109E8000D4F80330224ADBB2D37638BDD4F803309D
:109E90001F4ADBB2537638BDD4F803301C4ADBB21C
:109EA000137738BDD4F80330194ADBB2937638BD46
:109EB000D4F80330164ADBB2537738BDD4F8032008
:109EC000134B3CE7124BD4F803205A6238BD104BB9
:109ED000D4F803209A6238BD0D4BD4F80320DA621F
:109EE00038BD0B4BD4F803201A6338BD084BD4F8A7
:109EF00003205A6338BD064BD4F803209A6338BD5B
:109F0000034BD4F80320DA6338BD04223FE600BFD8
:109F1000F4050020554B2DE9F74F00241C60544BED
:109F2000544D1C60544B554EDFF874B12C631C60CB
:109F300085F8344005F1380705F10C0A05F14409AC
:109F40005FFA84F82421404605F046F9002304F81E
:109F50000B30337E4AF82400494A002B54D1494B38
:109F600049F8243045F8243042F824303B603B68FF
:109F700001932821404605F02FF9019B98473B6843
:109F8000B06229214046019305F026F9019B9847CC
:109F90003B68F0622A214046019305F01DF9019BC0
:109FA00098473B6830632B214046019305F014F934
:109FB000019B984757F8043B70632C21404601935E
:109FC00005F00AF9019B98470134032CB06306F1B0
:109FD0006406B5D12C4A00231946904642F8231056
:109FE0000133B3F5807FF9D1284CA37E43BBE37ED8
:109FF00053B3637DBBB3FEF7DBFDA0B3012385F84C
:10A000005C3003B0BDE8F08F214B49F82430214B80
:10A0100045F82430204B42F82430204BA6E7B919EC
:10A0200009EB0700042251440437FEF70BFF0C2F05
:10A03000F5D10C36FC2EDAD0002706F28C69EEE75B
:10A040000C26DFF860A0F7E74FF4FF6640F6D8076C
:10A05000A6F5FF613046042241440436FEF7F2FEC5
:10A06000BE42F5D1C5E70023C9E700BF8007002045
:10A070009C07002078F6FF1F800600209803002030
:10A08000C8F6FF1F3BF50000A00700200C80FF1F53
:10A090002BF5000033F500002FF5000037F5000028
:10A0A0005303002084060020014B93F85D007047A5
:10A0B00078F6FF1F70B5644E644B642505FB0065A0
:10A0C0000446A96A99420CD8EA6A9A4209D82A6BCE
:10A0D0009A4206D86A6B9A4203D8AA6B9A4240F217
:10A0E0008380642505FB046502220021204605F0DB
:10A0F000B3F8D5ED0A7AF8EE677A17EE900A07F012
:10A10000E3FB0022524B07F033FC4DA3D3E90023BD
:10A1100007F058FD07F03EFE28210246204605F0D4
:10A1200035F8D5ED0B7AF8EE677A17EE900A07F05E
:10A13000CBFB0022464B07F01BFC41A3D3E90023D5
:10A1400007F040FD07F026FE29210246204605F0D3
:10A150001DF8D5ED0C7AF8EE677A17EE900A07F045
:10A16000B3FB00223A4B07F003FC35A3D3E90023ED
:10A1700007F028FD07F00EFE2A210246204605F0D2
:10A1800005F8D5ED0D7AF8EE677A17EE900A07F02C
:10A190009BFB00222E4B07F0EBFB29A3D3E9002306
:10A1A00007F010FD07F0F6FD2B210246204604F0D3
:10A1B000EDFFA86B07EE900AF8EE677A17EE900AAB
:10A1C00007F082FB0022224B07F0D2FB1CA3D3E94D
:10A1D000002307F0F7FC07F0DDFD02462C212046A6
:10A1E000BDE8704004F0D2BF1A4E06EB840602228E
:10A1F000002105F03FF8336DA86A984728210246F0
:10A20000204604F0C3FF336DE86A984729210246CF
:10A21000204604F0BBFF336D286B98472A21024685
:10A22000204604F0B3FF336D686B98472B2102463C
:10A23000204604F0ABFF336DA86B9847CDE700BF15
:10A24000000000A2941AED4298030020FFFF3F0097
:10A250000000404278F6FF1FF7B5014C637801E03B
:10A2600078060020FF2B00F22F86DFE813F025028E
:10A27000380259026702720290029D02BF022D0647
:10A280002D062D062D06D302E502F60213031E034A
:10A29000270330033B0344034F0358035D0361036B
:10A2A000650369036D03710383032D062D062D06D7
:10A2B00090039E032D062D062D062D062D062D0638
:10A2C0002D062D062D062D062D062D062D062D06F6
:10A2D0002D06AC032D062D062D062D062D062D066A
:10A2E0002D062D062D062D062D062D062D062D06D6
:10A2F0002D062D062D062D062D062D062D062D06C6
:10A300002D062D062D062D062D062D062D062D06B5
:10A310002D062D062D062D062D062D062D062D06A5
:10A320002D062D062D062D062D062D062D062D0695
:10A330002D062D062D062D062D062D062D062D0685
:10A340002D062D062D06BB03C403CE03E103F40343
:10A35000FE030F0422042C0436044804580462044B
:10A360006C042D062D06760487049104A004AB042A
:10A37000AF042D062D062D062D06C0042D06CA0499
:10A38000D804EA042D06F5042D062D062D062D060B
:10A390002D062D062D062D062D062D062D062D0625
:10A3A0002D062D062D062D062D062D062D062D0615
:10A3B0002D060001090112011B012F0143014C016F
:10A3C00055015E0167017001790182012D062D069C
:10A3D0008B012D062D062D069401A6012D06C20126
:10A3E000CB01D401EB0101022D062D060A02130256
:10A3F000070510051D052D062D062D062D062B051E
:10A400003B0543052D061C022D062D062D062D06A7
:10A4100078059C052D06BA05C405CE052D062D062A
:10A420002D062D062D062D062D062D062D062D0694
:10A430002D062D062D062D062D062D062D062D0684
:10A440002D062D062D062D062D062D062D062D0674
:10A450002D062D062D062D062D062D062D062D0664
:10A46000DA052D06E4052D062D062D060106D4F885
:10A470000310A078C9B203B0BDE8F04004F054BBAB
:10A48000D4F80310A078C9B203B0BDE8F04004F0DE
:10A49000B7BBD4F80310A078C9B203B0BDE8F04050
:10A4A00004F0D2BBA07804F052FCD4F80310A378D7
:10A4B000C9B228B9184603B0BDE8F04004F002BCA8
:10A4C000184603B0BDE8F04004F0D0BBA07804F01B
:10A4D0003EFCD4F80310A378C9B228B9184603B0DB
:10A4E000BDE8F04004F00EBB184603B0BDE8F040F4
:10A4F00004F0D6BBD4F80310A078C9B203B0BDE80D
:10A50000F04004F0E5BAD4F80310A078C9B203B063
:10A51000BDE8F04004F09CBCD4F80310A078C9B2A8
:10A5200003B0BDE8F04004F04EBCD4F80310A078AE
:10A53000C9B203B0BDE8F04004F057BCD4F8031032
:10A54000A078C9B203B0BDE8F04004F02ABCD4F84A
:10A550000310A078C9B203B0BDE8F04004F057BCC6
:10A56000D4F80310A078C9B203B0BDE8F04004F0FD
:10A5700081BCD4F80310A078C9B203B0BDE8F040A4
:10A5800004F056BCD4F80310A078C9B203B0BDE8FB
:10A59000F04004F0FFBAD4F803000028C0F26D8444
:10A5A000A478B44B03EB84035B6C9847B24B6422F2
:10A5B00002FB0434206103B0F0BDD4F8030000288E
:10A5C000C0F25B84A378AC4A642101FB03231B7EA9
:10A5D000012B01D004F0ADFF0028D2BFA74AA84A42
:10A5E00092FBF0F21421A07803B0BDE8F04004F033
:10A5F000F7B9D4F80310A078C9B203B0BDE8F040B1
:10A6000004F010BBD4F80310A078C9B203B0BDE8C1
:10A61000F04004F09BBAD4F803000028C0F22D8467
:10A62000A378954A642101FB03231B7E012B01D0F3
:10A6300004F07FFF0028CABF914A904A92FBF0F2D3
:10A640001321D0E7D4F80310A078C9B204F0A1FC1C
:10A650000021A07804F0F8F9D4F803100246A0789D
:10A6600019B142F004020021BEE722F00402BBE768
:10A67000D4F80310A078C9B203B0BDE8F04004F0EC
:10A6800098BCD4F80310A078C9B203B0BDE8F0407C
:10A6900004F06DBCD4F80310A078C9B203B0BDE8D3
:10A6A000F04004F052BCD4F80310A078C9B203B053
:10A6B000BDE8F04004F025BCA078724A6023434313
:10A6C000D35CD4F803202BB9372103B0BDE8F040A8
:10A6D00004F05CBD6C4B53F820301A44F4E7A578C5
:10A6E000684A60236B43D35C23B9D4F8032021214B
:10A6F0002846EAE72121284604F06EFDD4F803300D
:10A70000C01A614B43F82500A5785021284604F073
:10A7100063FDD4F80330C01A5C4B43F825004AE7C8
:10A72000A5785B4BD4F8030001225A55514B03EB3B
:10A7300085035B6C984724210246D9E7A5784D4BE9
:10A74000D4F8030003EB85035B6C98472221024693
:10A75000CEE7A678474DD4F8030005EB8606736C68
:10A7600098470028B8BF4042F0602021A07804F04C
:10A7700033FD43077FF51FAFA678D4F8030005EB40
:10A7800086056B6C98472421024630469DE73A4A7D
:10A79000A078642303FB0023D4F803209A6203B05B
:10A7A000BDE8F040FFF786BCA578334B354AE0782A
:10A7B000642101FB053160236B434872D35C43B9CC
:10A7C0008A7A897D8DE803000621284604F0B4FCCE
:10A7D000F1E61021284604F037F9E37820F4F85226
:10A7E000DB0842EA032210212846FDE6A078224B2E
:10A7F000E278244C642101FB0031602343438A72D8
:10A80000E35C002B7FF4D7AE8C7D0194497A0091F4
:10A810000621DBE70121A07804F0DEFCD4F8033048
:10A8200020F00A02DF0748BF42F002029E0701D56E
:10A8300042F00802012175E00121A07804F0CCFC6F
:10A84000D4F8033020F00502DD0748BF42F00102D2
:10A850009807EFD542F00402ECE7D4F80320012A70
:10A8600000F20B83A3780449642000FB0313DA751C
:10A87000A1E600BF78F6FF1F98030020B500100086
:10A880000024F400C80400204003002058030020E6
:10A8900053030020A578B64BD4F8030003EB8503DF
:10A8A0005B6C98472521024622E7B24AA0786423D0
:10A8B00003FB0023D4F803201A6370E7AD4AA078A5
:10A8C000642303FB0023D4F80320DA6267E7A5784A
:10A8D000A74BD4F8030003EB85035B6C9847272153
:10A8E000024605E7A34AA078642303FB0023D4F8BB
:10A8F00003205A6353E7A5789D4BD4F8030003EB7C
:10A9000085035B6C984726210246F1E6994AA078B8
:10A91000642303FB0023D4F803209A633FE7D4F8B1
:10A9200003202D21A078D0E6D4F803202E21F9E7CA
:10A93000D4F803202F21F5E7D4F803203021F1E7E4
:10A94000D4F803203321EDE7D4F803203421E9E7DC
:10A950000121A07804F040FCD4F8033020F0C002BC
:10A96000D90748BF42F040029B077FF563AF42F032
:10A9700080025FE70121A07804F02EFCD4F80330B8
:10A980001B0220F4407203F440731A4352E7012182
:10A99000A07804F021FCD4F8033020F01002002B42
:10A9A0003FF448AF42F0100244E70121A07804F0E0
:10A9B00013FCD4F8033020F02002002B3FF43AAF10
:10A9C00042F0200236E7A0786B4A60234343D35C11
:10A9D000002B3FF4F0ADD4F8031003B0BDE8F04015
:10A9E00002F02EBBA078644BD4F80320602101FB59
:10A9F00000335A6069E66049A078D4F803206023E8
:10AA000003FB001361219A605FE6A0785A4A602335
:10AA100003FB0023D4F803201A731C2104F0DCFB91
:10AA2000D4F80320C0F3080040EA02421C2179E771
:10AA3000A078514A602303FB0023D4F80320DA8175
:10AA40001C2104F0C9FBD4F8033000F47F02C3F3E7
:10AA500008031A43EAE74849A078D4F803206023A2
:10AA600003FB001359211A612FE6A078D4F80320C4
:10AA7000414C60234343E118E35CD2B20A75002BDA
:10AA80003FF499AD8B7D01924A7D0FE0A078D4F818
:10AA90000320394C60234343E118E35CD2B24A758A
:10AAA000002B3FF488AD8B7D097D0191009200223F
:10AAB000AEE63149A078D4F80320602303FB0013ED
:10AAC0005A211A6201E62C49A078D4F803206023A9
:10AAD00003FB00135B215A62F7E5A0782649D4F8FE
:10AAE0000320602303FB0013D1B29A62C2F3072252
:10AAF00093F82C300191009200225D2166E6A07847
:10AB00001D49D4F80330602202FB0012D362926A1E
:10AB1000D1B2C2F3072201910092DBB2ECE71649F1
:10AB2000A078D4F80320602303FB00135E211A638E
:10AB3000CBE51149A078D4F80320602303FB001370
:10AB400018219A61C1E50C49A078D4F8032060234C
:10AB500003FB00131921DA61B7E50749A078D4F89F
:10AB60000320602303FB00135C215A63ADE500BFA3
:10AB700078F6FF1F98030020C8040020B449A0788D
:10AB8000D4F80320602303FB00135F219A639CE544
:10AB9000A078D4F80330AE4C60224243A118A25CE6
:10ABA000DBB28B75002A3FF406AD0A7D6BE7D4F863
:10ABB0000330022B00F26181A278A64B1344E278A5
:10ABC0001A76F8E4D4F803202021ABE6D4F8031079
:10ABD0009F48A278012905D19F4B99546023534384
:10ABE000C154E8E4602353430022C254E3E498498B
:10ABF000A078D4F80320602303FB00135221DA630A
:10AC000063E5934AA078E178602303FB00235A6C44
:10AC100083F84010019193F8413000930CE0A07844
:10AC20008B4AE178602303FB002383F841105A6CC0
:10AC300093F840308DE80A00D3B26321C2F30722B3
:10AC4000C4E58349A078D4F80320602303FB0013F4
:10AC50005A6493F84010DDE7D4F80330082B00F273
:10AC60000C810A21A07804F0B7FAD4F8033020F060
:10AC70000F02C3F108031A430A2153E6774AA37867
:10AC8000642101FB0323D4F803201A7293E4A5780E
:10AC9000704AD4F8030002EB8502536C9847642392
:10ACA0006B436E4AD05086E4A5786A4BD4F8030013
:10ACB00003EB85035B6C9847684B642202FB053508
:10ACC000686078E4A078654B614AE478642101FB10
:10ACD0000031602343438C75D35C002B7FF46BAC55
:10ACE0008A7A92E5D4F80310A07803B0BDE8F0406A
:10ACF00003F0BEBDA078594ED4F80320642505FBAF
:10AD000000618B8F9A423FF456AC60234343504F0F
:10AD1000FB5C03BB0C238A87009392B204230A21B5
:10AD200004F0B6FAA07805FB00635421DA69002A22
:10AD3000B8BF524204F02AFAA07805FB0065EB691F
:10AD4000002B4FF000524FF007017CDA03B0BDE852
:10AD5000F04004F081BA0622414B1A702BE4A5782A
:10AD60003B4A404E60236B43D75C97B15021284645
:10AD700004F032FAD4F80330C01A46F82500A5785A
:10AD80002121284604F028FAD4F80330C01A364BA3
:10AD9000C3E4D4F803205021284604F0F7F9A3783F
:10ADA00046F8237007E4A0782C4ED4F803206425DD
:10ADB00005FB0063DB699A423FF4FDAB602343432C
:10ADC0002349CB5C002BC6D1002AB8BF5242542184
:10ADD00004F0DCF9A078D4F8033005FB0065EB61E2
:10ADE000AEE71E49A078D4F80320642303FB0013C8
:10ADF00053211A6269E4194AA378642101FB0323F1
:10AE0000D4F803205A62FFF7D6BB1449A078D4F8CF
:10AE10000320642303FB001315219A82134B5A432A
:10AE200053E40E4AA378642101FB0323E27883F8FC
:10AE30003E20FFF7C0BBD4F80310A0784FF080523B
:10AE400009B1002182E703B0BDE8F04004F012BA76
:10AE5000C804002078F6FF1F530300209803002049
:10AE600094070020580300204003002000710200D6
:10AE7000D4F803301BB1012B12D004226CE7A17867
:10AE80001248642202FB01021148137600EB810292
:10AE9000104B536440F8213013659363FFF78BBB6D
:10AEA000A2780A48642101FB02010B480B7608498D
:10AEB00001EB82035864094841F82200084A1A65E8
:10AEC000084A9A63FFF777BB032245E798030020FF
:10AED00078F6FF1F3BF500002BF5000033F500006E
:10AEE0002FF5000037F500002DE9F04FC54EC64F95
:10AEF00032787A7064233B70212AD6F803307B6065
:10AF000085B034463D4601F05A8100F2C3800E2AD6
:10AF100000F0138639D8072A00F03F8414D8032A9A
:10AF200000F0518208D8012A00F09B81022A00F02B
:10AF3000F38102232B70E7E1052A00F02B8440F215
:10AF40007682FEF7ABF8DFE10A2A00F02C8407D8FE
:10AF5000082A00F02584092AEBD1FEF7FDFDD3E194
:10AF60000C2A00F0A58540F28E85B078022800F208
:10AF7000D0817378012B00F0B085C0F0AB85022B37
:10AF800000F0C48503233B70BEE1182A00F030872F
:10AF90002BD8142A00F07A8615D80F2A00F0EC85F9
:10AFA000132AC6D17178994A092900F24386DFE84D
:10AFB00011F03E064A064D06500654065B065E0634
:10AFC000610664065906162A00F00E8740F27F8655
:10AFD0008F4A116E072900F29781481C02EB81010C
:10AFE0001066106B486613638EE11C2A00F0FA8726
:10AFF00022D81A2A00F01A8740F20787844D95F864
:10B00000342072B95E1C04BF804B1B680A20584371
:10B01000C5F88800FDF730FB0123C5F88C0085F8E2
:10B0200034306378042B00F26F81DFE813F01007EF
:10B0300051077F07AD0726071F2A01F0088001F29C
:10B0400064801E2A7FF475AF7278142A00F22A8574
:10B05000B078022800F2CC8702EB42046D4D044424
:10B0600045F824306C4B9B7E002B00F04D81002A6C
:10B0700000F04A81032111FB02010C23013A5A43DB
:10B0800002F5D363042205EB810102FB0030FDF7DA
:10B09000A0FE39E1802A01F07D8144D8402A01F0E8
:10B0A000528129D8242A01F0E8800CD8222A01F004
:10B0B000DC80232A7FF43DAF544B1B68C6F8033075
:10B0C000FEF74AFD20E1262A01F01581C1F0088132
:10B0D000272A7FF42EAFB278022A00F21A81737801
:10B0E000142B00F2DF8403EB43031344474A116837
:10B0F000484A42F8231007E1442A01F0308107D87A
:10B10000422A01F0288141F2228101F044FFFBE054
:10B11000462A01F03B81C1F03581472A7FF409AF0F
:10B1200001F03DFFF0E0872A01F0CD8146D8832A67
:10B1300001F04E810AD8812A01F03281822A7FF4FF
:10B14000F8AE334B022283F85C20DDE0852A01F063
:10B150007281314A41F25C813049314C01250D70D8
:10B16000B3F5805F9178217081F06B81127D12EAD6
:10B17000050641F06681184602A9FDF787FE9DF895
:10B18000083063709DF80930A3709DF80A30E370B1
:10B190009DF80E3023719DF80D3063719DF80C30D1
:10B1A000A3719DF80B30E37126722B46E15C227A85
:10B1B00001330A44082B2272F8D1A5E08C2A01F051
:10B1C000CA813BD8892A01F0AB81C1F044818A2A27
:10B1D0007FF4AFAE7278134B002A41F0B9811A7038
:10B1E000114AE37813700A4A92F874110F4A1170E9
:10B1F0000F4900220A700F490A700F4A11780B4359
:10B20000137081E07806002094070020800700205A
:10B2100078F6FF1F840600200C80FF1F84070020A3
:10B220008507002038030020640300204406002026
:10B23000560300207406002039030020F22A01F092
:10B240000F82FF2A01F051828D2A7FF472AE72784C
:10B25000032A01F2EB81DFE812F0BE09A509D70944
:10B26000E509B378022B54D8A64FDFF8B0A2DFF877
:10B27000B0B20026B846A378F5B2AB4209D064223A
:10B2800002FB038393F83E30CBB397F83E209A42FB
:10B2900035D1284601F002FF9B4A00234FF00109F7
:10B2A000B35406F80A304FF0006206F80B90494696
:10B2B000284603F0D1FFFA7D4ABB4A4620212846A2
:10B2C00003F064FF914BD4F8030053F826309847FD
:10B2D00024210246284603F059FF4FF080520721EF
:10B2E000284603F0B9FF4FF000620721284603F01B
:10B2F000C1FF4FF000620121284603F0BBFF013679
:10B30000032E07F16407B6D105B0BDE8F08F022225
:10B31000D4E704232B70F7E7B378022BF9D8794FE1
:10B32000DFF8F8A1DFF8F8B10026B846A378F5B247
:10B33000AB4209D0642202FB038393F83E30D3B3BF
:10B3400097F83E209A4236D1284601F0A7FE6E4A71
:10B3500000234FF00109B35406F80A304FF00062A1
:10B3600006F80B904946284603F076FFFA7D42BB6B
:10B370004A462021284603F009FFD4F80300634B16
:10B38000404253F82630984724210246284603F0CD
:10B39000FDFE4FF080520721284603F05DFF4FF07D
:10B3A00000620721284603F065FF4FF0006201218B
:10B3B000284603F05FFF0136032E07F16407B5D17D
:10B3C000A2E70222D5E7B378022BA2D84D4FDFF8CF
:10B3D00050910026B8464FF0010AA378F5B2AB426F
:10B3E00009D0642202FB038393F83E30BBB197F887
:10B3F0003E209A4213D1284602F0E8FEFB7D06F873
:10B4000009A093B901222021284603F0BFFE284657
:10B410000022242103F0BAFE284601F03FFE013647
:10B42000032E07F16407D8D16EE70222EBE7B0786C
:10B43000022803D97278022A7FF466AF6278012A63
:10B4400000F0D4806ED3022A7FF45EAF142B3FF756
:10B4500060AF020640F14F812B4FDFF8C080DFF86C
:10B46000A4900025A3782B41DB0747D5EEB23046E8
:10B4700001F014FE0023EB5505F80830642303FBAC
:10B480000593DB7D002B40F028810522DFF890A09A
:10B490002021304603F07AFE15F80A304BB11C4BE0
:10B4A000242153F82520304603F070FE002305F8D0
:10B4B0000A304FF080520721304603F0DBFE4FF098
:10B4C00000620721304603F0C7FE6023114A6B4338
:10B4D0009B5C114A002B40F00281D4F8033003EB4F
:10B4E00043032B4452F823203721304603F04EFE0D
:10B4F0004FF000620121304603F0BCFE0135032D00
:10B50000B0D101E79803002090030020BCF6FF1F94
:10B5100084F6FF1FC804002084060020500300208A
:10B5200053030020BC4FDFF800A3DFF808B3DFF8B7
:10B53000FC820025B946A378AB420AD0642202FB04
:10B54000039393F83E30002B43D097F83E209A4265
:10B550003FD1EEB2304601F0A1FD002305F80A30DC
:10B5600005F80B304FF000620121304603F074FE05
:10B57000FB7DA3BB05222021304603F007FE15F812
:10B5800008304BB1A54B242153F82520304603F059
:10B59000FDFD002305F808304FF0805207213046AA
:10B5A00003F068FE4FF000620721304603F054FEBE
:10B5B00060239B4A6B439B5CD4F803208BB93721F3
:10B5C000304603F0E3FD4FF000620121304603F006
:10B5D00051FE0135032D07F16407ACD194E6062234
:10B5E000C9E7904B53F825301A44E8E7DFF8288282
:10B5F000DFF840A2DFF84CB20025C146A378AB4289
:10B600000AD0642202FB039393F83E30002B51D002
:10B6100098F83E209A424DD1EEB2304601F03EFD00
:10B62000814A0023AB5405F80A304FF00062012133
:10B63000304603F011FE98F817306BB9052220212F
:10B64000304603F0A3FD15F80B30012B38D005D39D
:10B65000022B37D0002708E00622F0E737213046DA
:10B6600003F0BAFDD4F803700744704BEA5C52B1A2
:10B670006A4A019352F825202421304603F086FDC2
:10B68000019B0022EA544FF080520721304603F01C
:10B69000F1FD4FF000620721304603F0DDFD3A4630
:10B6A0003721304603F072FD4FF000620121304631
:10B6B00003F0E0FD0135032D08F164089ED123E677
:10B6C0002121CCE75021304603F086FD584B53F83A
:10B6D0002570C71BD4F80300C6E70622D6E6D4F8C7
:10B6E000033003EB43032B4452F823204D4B53F814
:10B6F00025301A44F8E602283FF60BAE01F0CEFCE6
:10B70000A078494A002313544A4A1354424A6423F6
:10B7100003FB0023DB7D002B35D10522202103F024
:10B7200035FD424DA0782B5C4BB1434B03EB8003BE
:10B730002421DA6803F02AFDA3780022EA544FF0AE
:10B7400080520721A07803F095FD4FF00062072199
:10B75000A07803F081FDA078314A60234343D15C97
:10B76000D4F80330354A03EB4303034452F8232053
:10B7700059B9372103F00AFD4FF000620121A0788A
:10B7800003F078FDC0E50622C8E7264B53F82030C9
:10B790001A44EEE7FEF760FDB6E5FDF771FCB3E590
:10B7A000FDF76EFCB0E5B378022B00F0CE80032BE2
:10B7B00000F0D080002B40F05F817378502B00F0B8
:10B7C0009A8041D8462B00F0878010D8422B7DD03C
:10B7D00006D8402B60D0412B74D003232B7060E03F
:10B7E000442B76D0452BF8D1154B5B796CE04B2B75
:10B7F00078D009D8472B72D0492BEED1104BDB7D86
:10B80000003318BF01235FE04D2B71D06DD34F2B58
:10B81000E3D10B4B5B7E57E09803002084F6FF1FBB
:10B82000C8040020400300209003002053030020A0
:10B83000580300205003002078F6FF1F84060020E4
:10B840000C80FF1F90F6FF1F802B63D012D8532B64
:10B8500057D006D8512B51D0522BBED1A04B1B6ACA
:10B8600032E0552B53D04FD3562BB6D19C4B93F887
:10B87000243029E0832B58D006D8812B4ED0822B40
:10B88000ABD1984B1B6B1FE0852B53D04FD3FF2BB5
:10B89000A3D1954B1B78B3E745F2FF70FDF7C0FAD3
:10B8A0007860924B1B78002B3FF42EAD904B6A686A
:10B8B0001A60904B002A40F0E1801A6842F00802BA
:10B8C0001A6021E5864B1B786B60EAE7844B5B7856
:10B8D000FAE7834BDB69F7E7814BDB68F4E7804BE2
:10B8E0009B68F1E77E4BDB78EEE77D4B9B78EBE7DF
:10B8F0007B4B5B7DE8E77A4B9B7DE5E7784B1B7DD7
:10B90000E2E7774B1B69DFE7754B9B7EDCE7744B07
:10B91000DB7ED9E7734B93F85C30D5E7714B93F836
:10B920005C301E1F73427341CEE76E4BD2E7724B01
:10B930001B68C9E76B4A7148136A43F2390100FB7F
:10B940000313136223F00043BEE772786C4B53F885
:10B950002230B9E773782E2B3FF63FAF01A252F8A1
:10B9600023F000BF21BA000025BA00002BBA000066
:10B97000DBB70000DBB70000DBB70000DBB700007F
:10B98000DBB70000DBB70000A3B80000A3B80000DD
:10B99000A3B80000DBB70000DBB70000DBB7000096
:10B9A000DBB70000DBB70000DBB70000DBB700004F
:10B9B000DBB70000DBB70000DBB70000DBB700003F
:10B9C000DBB70000DBB70000DBB70000DBB700002F
:10B9D0002FBA000035BA000039BA00003DBA0000A5
:10B9E00043BA000047BA0000DBB70000DBB7000035
:10B9F000DBB70000DBB70000DBB70000DBB70000FF
:10BA00004DBA000051BA000057BA00005DBA0000FC
:10BA100063BA000067BA00006DBA000073BA000094
:10BA2000384B85E7374B5B684EE7364B58E7354B6D
:10BA30001B7E49E7334B6BE7324BEBE6314B1B7F09
:10BA400042E7304B61E72F4B5B7F3DE72D4B06E72D
:10BA50002C4B5B6A38E72B4B9B6A35E7294BDB6A3B
:10BA600032E7284B0EE7274B5B6B2DE7254B9B6B93
:10BA70002AE7244BDB6B27E70423AFE61A6822F0A2
:10BA800008021A6040E4B378022B0ED17078372890
:10BA900008D800F5FF701C49800004220144FDF71E
:10BAA00098F931E403232B702EE404233B702BE43C
:10BAB000B378022B0BD170783728F3D800F5FF70DC
:10BAC0001149800004220144FDF7BCF91CE4042361
:10BAD0003B7019E402F072FB16E402F077FB13E40A
:10BAE0000C80FF1F78F6FF1F8E0700208F070020B5
:10BAF0008007002080060020900700206D4EC64180
:10BB0000A0070020F4050020A8FFFF1F02F066FB3D
:10BB10009E4B78601B78002B3FF4F6AB9C4B186073
:10BB20009C4B1A6820B942F008021A60FFF7ECBB80
:10BB300022F008021A60FFF7E7BBB278022A17D199
:10BB40007078072808D81BB9FCF75EFFFFF7DCBB4D
:10BB5000FCF746FFFFF7D8BBFF287FF4D5AB5D1C91
:10BB60000ABF8B4BD8B21878FCF762FFFFF7CCBB4B
:10BB700004233B70FFF7C8BBB378012B2AD023B155
:10BB8000022B4AD004233B700FE07078082803D8BA
:10BB9000FCF75FFF686008E00A2816D17E4B1B693E
:10BBA00083F40073C3F340237B60784B1B78002B36
:10BBB0003FF4AAAB764B6A681A60764B8ABB1A6868
:10BBC00042F008021A60FFF79FBBFF28EDD1FCF797
:10BBD00077FFDFE77078092802D002F089FBD9E708
:10BBE0000020FCF785FF04460120FCF781FF064694
:10BBF0000220FCF77DFF8642D4BF002301239C4234
:10BC000009DD331C18BF01231BB986423446B8BF77
:10BC100004466C60C9E7031CF4E77078FCF732FF58
:10BC2000B8E71A6822F008021A60FFF76DBB1068C7
:10BC3000184410601268574B12BB1A6842F0080291
:10BC40001A60FFF761BB1068C01AF2E7106858432A
:10BC5000EFE7106890FBF3F0EBE7116891FBF3F06E
:10BC600003FB10131360E5E710681840E1E7106864
:10BC70001843DEE710685840DBE71368DB43F1E761
:10BC80001A6822F008021A60FFF73EBB404A1168AA
:10BC9000404A8B4213680BDA23F0030343F004039A
:10BCA0001360136871B943F008031360FFF72CBBEE
:10BCB0000BBF23F0060323F0050343F0010343F019
:10BCC0000203EDE723F008031360FFF71DBB727852
:10BCD0000C2A3FF619ABDFE802F0071019222B34CB
:10BCE0003E4750636C757E002A4A126814077FF540
:10BCF0000BAB2A4A1363FFF707BB264A12681007EB
:10BD00003FF502AB254A1363FFF7FEBA214A1268DA
:10BD1000D1077FF5F9AA214A1363FFF7F5BA1D4A47
:10BD20001268D2073FF5F0AA1C4A1363FFF7ECBA7A
:10BD3000184A126857077FF5E7AA184A1363FFF7F6
:10BD4000E3BA144A126812F0050F3FF4DDAA134A51
:10BD50001363FFF7D9BA0F4A126896077FF5D4AA82
:10BD60000E4A1363FFF7D0BA0A4A126895073FF4E8
:10BD7000CBAA0A4A1363FFF7C7BA064A1268D40669
:10BD80007FF5C2AA054A1363FFF7BEBA8F070020EA
:10BD9000800700208006002080F00F4078F6FF1F0B
:10BDA000B94A126890067FF5AFAAB84A1363FFF745
:10BDB000ABBAB54A126851067FF5A6AAB34A136317
:10BDC000FFF7A2BAB04A126812067FF59DAAAF4AE1
:10BDD0001363FFF799BAAC4A1268D7057FF594AAA6
:10BDE000AA4A1363FFF790BAA84A1363FFF78CBA05
:10BDF000A64A136E002B3FF487AA013B136602EBA1
:10BE000083035B6E1363FFF77FBA73782E2B04D81E
:10BE10009F4A0121D154FFF777BAFF2B7FF442AE3E
:10BE20009A4B012283F88420FFF76EBA73782E2B89
:10BE300004D8974A0021D154FFF766BAFF2B7FF44C
:10BE400031AE924B002283F88420FFF75DBAFCF7F5
:10BE500013FCD5F88C30C01A0028D5F88830B8BF4C
:10BE60004042984295BF2B6B002303F1FF3385F8C6
:10BE7000343098BF2B63FFF747BAA07802F0AEF9D1
:10BE800040B9814A85F83400136823F01003136029
:10BE9000FFF73ABAD5F88830ABB1FCF7EDFBD5F82F
:10BEA0008C30C01A0028D5F88830B8BF404298427C
:10BEB00009D9754A002385F83430136843F010031C
:10BEC0001360FFF721BA2B6B013B2B63FFF71CBA02
:10BED000A0780F2103F080F910F0010409D06A4A1C
:10BEE000002385F83430136823F010031360FFF744
:10BEF0000BBAD5F88830A3B1FCF7BEFBD5F88C306F
:10BF0000C01A0028D5F88830B8BF4042984208D9F6
:10BF10005D4A85F83440136843F010031360FFF75F
:10BF2000F3B92B6B013B2B63FFF7EEB9A0780F2120
:10BF300003F052F910F0800409D0534A002385F829
:10BF40003430136823F010031360FFF7DDB9D5F820
:10BF50008830A3B1FCF790FBD5F88C30C01A0028CC
:10BF6000D5F88830B8BF4042984208D9464A85F88B
:10BF70003440136843F010031360FFF7C5B92B6B0F
:10BF8000013B2B63FFF7C0B9A0780F2103F024F920
:10BF900010F4807409D03C4A002385F834301368CB
:10BFA00023F010031360FFF7AFB9D5F88830A3B1C1
:10BFB000FCF762FBD5F88C30C01A0028D5F8883021
:10BFC000B8BF4042984208D92F4A85F834401368D8
:10BFD00043F010031360FFF797B92B6B013B2B6302
:10BFE000FFF792B9294B002283F85C20FFF78CB948
:10BFF000FF287FF48EA9274E3AB300254FF003089F
:10C000000C27607818FB00510138784300F5D360A5
:10C0100000EB8500042206EB81010135FCF7D9FE17
:10C02000032DEED1FFF770B9291978190422314494
:10C030000435FCF7CEFE0C2DF6D10C34FC2C3FF46D
:10C0400063A9002504F28C67EEE70C24F9E7737806
:10C05000142B3FF627ADB278022A27D803EB43030F
:10C0600013440C4A52F823200B4B7A601B78002BA8
:10C070003FF44AA9094B1A60034B8AB91A6842F087
:10C0800008021A60FFF740B98006002078F6FF1F0B
:10C0900045060020840600208F070020800700202E
:10C0A0001A6822F008021A60FFF72EB9FF2A7FF4FF
:10C0B00030A9AD4E3BB300254FF003080C27607844
:10C0C00018FB00510138784300F5D36000EB850080
:10C0D000042206EB81010135FCF7B4FE032DEED1FD
:10C0E000FFF712B961197819042231440435FCF7BD
:10C0F000A9FE0C2DF6D10C34FC2C3FF405A900252B
:10C1000004F28C67EEE70C24F9E77678142E3FF6FC
:10C11000C9ACA77838062AD5934FDFF8508200259E
:10C12000A3782B41D90709D566782121E8B203F01D
:10C1300053F806EB46062E4447F8260098F81A30C6
:10C1400083B1637873B1032111FB03510C20013BD0
:10C15000584300F5D360042207EB810100EB850012
:10C16000FCF737FE0135032DDAD1FFF7CDB8022FEA
:10C170003FF6CFA82121384603F02EF87B4B7A4DAD
:10C180009B7E06EB46063E4445F82600002B3FF416
:10C19000BBA86278002A3FF4B7A8A078032111FB5E
:10C1A00002010C23013A534303F5D363042205EB48
:10C1B000810102FB0030FCF70CFEFFF7A5B8727896
:10C1C0006B4B0A2A0CD8DFE802F006151A1F252D42
:10C1D00032373C41450067491A6809680A441A60C9
:10C1E0001A68654B002A3AD11A6842F008021A60B0
:10C1F000FFF78AB85F491A680968521AEFE75D4A83
:10C20000196812684A43EAE75A491A68096892FBB2
:10C21000F1F2E4E7574A1868116890FBF1F201FB6C
:10C220001202DCE753491A6809680A40D7E7514906
:10C230001A6809680A43D2E74E491A6809684A40F1
:10C24000CDE74C490A68D2430A60C9E71968494AF0
:10C250001160C5E7474A196810681860F8E71A685E
:10C2600022F008021A60FFF74FB8414B1B68C6F86E
:10C270000330FDF7F1FFFFF747B87378052B3FF662
:10C2800043A8DFE803F0030A11181F263A4A13688F
:10C2900003F00F031360FFF737B8374A136823F032
:10C2A00010031360FFF730B8334A136823F02003FC
:10C2B0001360FFF729B8304A136823F04003136076
:10C2C000FFF722B82C4A136823F080031360FFF7AE
:10C2D0001BB8294A136823F480731360FFF714B85E
:10C2E00071782E293FF6DEAB244A02EB8102C2F8B8
:10C2F0009030FFF709B8214B1D4AD3F84C1111605B
:10C300001C4AD3F850111160D3F854211A631A4A09
:10C31000D3F858111160D3F85C2183F83420D3F896
:10C320006021C3F88C20D3F86421C3F8882093F8E7
:10C330006811134A505C08B101205054002283F860
:10C340006C21FEF7E1BF00F011FEFEF7DDBF00F04B
:10C350000EFEFEF7D9BF00F01DFEFEF7D5BF00F0C0
:10C360001BFEFEF7D1BF00BF840600200C80FF1F1C
:10C37000800700209C0700208006002078F6FF1F21
:10C380004506002000F009FEFEF7BEBF00F006FEE5
:10C39000FEF7BABFA74B002283F85C20FEF7B4BFBC
:10C3A00072782AB1012A09D003233B70FEF7ACBF93
:10C3B000A04B012283F85C20FEF7A6BFB3F5805F97
:10C3C000BEF4A7AF9B4981F85C200B63FEF79CBFCE
:10C3D000984A9948002382F8843082F86C3102F13F
:10C3E00090044FF0FF35194644F82350C1540133EF
:10C3F0002F2BF9D1914B82F85C101960904B11638F
:10C400001960904B116682F834101960FEF77CBFFA
:10C41000127D92070BD4B3F5805FBEF47AAF854AE4
:10C42000042182F85C10C2F87031FEF76DBF08235A
:10C430003B70FEF769BF7F4B002283F85C20FEF75C
:10C4400063BF2B460022E2540133082BFBD1237833
:10C450002372FEF759BF7378012B19D005D3022B35
:10C460001FD003233B70FEF74FBF774B01221A709A
:10C47000764B774A9B781370764B19680023013905
:10C48000013311F8010FD054082BF9D1FEF73CBF4E
:10C490000C22FA717B71F2220923BA713B71FEF70B
:10C4A00033BF694B6C4801221A70684B684A9B780D
:10C4B0001370002301331918082B11F8091CD154EB
:10C4C000F8D1FEF721BF7378032B3EF61DAFDFE8EE
:10C4D00003F002101D22574B93F85C20FA7193F879
:10C4E0003420D3F87031BA711A0A7A713B71FEF7B1
:10C4F0000BBF504B93F85C20FA7193F834201B6B00
:10C50000BA711A0A7A713B71FEF7FEBE4B4B1B687B
:10C510007B60FEF7F9BE4A4B1B687B60FEF7F4BEFA
:10C520007278002A7EF4F0AEB17800297EF4ECAE89
:10C5300040F2D24293427EF4E7AE45F2FF70FCF740
:10C5400036FCFCF7B1FC0120FCF772F9FEF7DCBE0B
:10C550000122FEF744BE74782CB1012C13D00323C2
:10C560003B70FEF7D1BE042202A945F2FB70FCF736
:10C5700069FC029BD6F803209A4206BF01237B6028
:10C580007C60FEF7C1BEB3782A2B07D10422334961
:10C5900045F2FB70FCF71DFCFEF7B6BE03233B70B3
:10C5A000FEF7B2BE234CD4F87801002104F5BE7228
:10C5B00081423EF4A9AE52F821509D4201F101059D
:10C5C00020D102EB8503043B0138814214D3C4F827
:10C5D0007801FEF799BE174AD2F8781109299DBF54
:10C5E000481CC2F8780102EB8102092394BFC2F80B
:10C5F0007C313B70FEF788BE53F8042F43F8042CBF
:10C600000131E2E72946D3E70A4A0023C2F878312C
:10C61000194602F5BE7242F8231001330A2BFAD1F3
:10C62000FEF772BE0A237B60FEF76EBE03233B70EB
:10C63000FEF76ABE78F6FF1F45060020800700203F
:10C640009C07002080060020840700200C80FF1F2C
:10C65000850700200880FF1F008000007B06002067
:10C660007378812B7EF455AEB378922B7EF451AE65
:10C67000B379A32B7EF44DAE7379B42B7EF449AE1F
:10C680003379C52B7EF445AEF378D62B7EF441AEDC
:10C69000FCF7C9FAFBF7F0FF0446FBF7EDFF001BC0
:10C6A0000028B8BF4042B0F57A7FF6DBFCF7BEF851
:10C6B000134B00221A604FF0FF32C3F87021C3F809
:10C6C0007022C3F87421C3F87422C3F87821C3F828
:10C6D0007822C3F87C21C3F87C220A4B0A4A1A60EC
:10C6E0000120FCF7A5F8FEF70FBE40F2D2429342BC
:10C6F0007EF40AAE054B012283F8A421FEF704BEA6
:10C7000010E000E00080FF1F7856341278F6FF1F1B
:10C71000F7B50F4C07460E4694E803008DE803007A
:10C720000C49C1F803300C4B8A7000220F704E7018
:10C730001A70FEF7D9FB094A217882F85D109DE84E
:10C740000300636884E80300184603B0F0BD00BF2F
:10C7500094070020780600208F07002078F6FF1F3E
:10C76000F7B504461F4A63781370A3785370E378D3
:10C7700093702379937163795371A3791A4D13716F
:10C78000E379D3700E4695E80300184B00221A7027
:10C790008DE80300FEF7A8FB154B1A786F462B4671
:10C7A0009AB9327072702A78B2706A78F270EA7947
:10C7B0003271AA7972716A79B2712A79F27197E845
:10C7C000030083E8030003B0F0BD012AF7D1094854
:10C7D000721EF11D10F8014F02F8014F8A42F9D183
:10C7E000EDE700BF78060020940700208F070020A7
:10C7F00084070020850700202DE9F043994B9A4CCF
:10C800001B788FB06BB1994B1B78063BDBB2192BB1
:10C8100004D8974A22FA03F3D90702D4002384F8F4
:10C82000743194F87431934E5A1E012A51D89249AA
:10C83000012BCA68079214BF082307238DF818300C
:10C84000327894F8A5318DF8193000238DF81A301C
:10C85000002A33D18B688DF82030884B8DF8272043
:10C8600019788DF8211059788DF82210D9798DF822
:10C87000231099798DF8241059791B798DF825109A
:10C880008DF8263006A801F051FE002800F01F8325
:10C890007B4B1A789846002A00F01E81794B7A4F1C
:10C8A0001B78013B062B00F21381DFE813F0F10047
:10C8B000F10058011101110111017F01012AE1D19B
:10C8C0007248013306AA1A44195CD171082BF8D1B9
:10C8D000D8E7032B3DD1337883BBDFF89C81674FCA
:10C8E00098F8020098F801503B7805441D447B7885
:10C8F0001D44FB791D44BB791D447B791D443B7964
:10C900001D44FBF7F3FE98F80100FBF7EFFE3878C3
:10C91000FBF7ECFE7878FBF7E9FEF879FBF7E6FE2B
:10C92000B879FBF7E3FE7879FBF7E0FE3879EDB2F2
:10C93000FBF7DCFE2846FBF7D9FEA9E7012BA7D1C0
:10C94000524F0025785D0135FBF7D0FE092DF9D156
:10C950009EE7042B2BD1484FDFF82081B8787D78F3
:10C96000002301220544154488F8013088F800208E
:10C97000C8F80430FBF7BAFE7878FBF7B7FE98F8F2
:10C980000000FBF7B3FE98F80100FBF7AFFE98F844
:10C990000700FBF7ABFE98F80600FBF7A7FE98F838
:10C9A0000500FBF7A3FEEDB298F80400C0E7072BE3
:10C9B00037D1337853BB304B9F7893F801802F4B9E
:10C9C0008DF800701D785878D9798DF80250474459
:10C9D0003D449A798DF80300284493F805C08DF8FA
:10C9E0000410014493F804E08DF805200A440CEB90
:10C9F000020373448DF801808DF806C08DF807E0BE
:10CA00008DF808306846FCF70BF941E7012BF9D1A6
:10CA10001E4900235A5C0DF803200133092BF9D17C
:10CA2000F0E7082B7FF434AF144A134900230120A8
:10CA30005370107053608A7849788DF800200A444A
:10CA400002448DF801108DF802008DF803308DF846
:10CA500004308DF805308DF806308DF807308DF8EC
:10CA60000820CFE78E07002078F6FF1F7806002009
:10CA700011020002840700200C80FF1F9407002091
:10CA8000740600204406002056030020850700207D
:10CA9000AE4A397893688DF8303080238DF8313084
:10CAA0008A238DF8323000238DF833308DF83430FE
:10CAB0008DF835308DF836108DF8293007218DF836
:10CAC0002A300AA8D3688DF828100B9301F02EFDA8
:10CAD00000233B7088F80030002384F874313370F1
:10CAE00094F8A43113B10120FBF7A2FE06A801F0CF
:10CAF000A9FC0646002800F04181954B9DF82020B6
:10CB00001A709DF821205A709DF822209A709DF885
:10CB100023209A719DF824205A719DF825201A71BE
:10CB20009DF82620DA709DF8193084F8A531FBF7BE
:10CB3000A3FD884B1860884B00221A709DF81830AE
:10CB4000072B0CBF0123022384F8743194F85C3066
:10CB50005A1E012A4AD9052B48D0012247E0DFF8A6
:10CB6000EC913B7899F8020099F8015005440A3598
:10CB70001D44FBF7BBFD99F80100FBF7B7FD8020D2
:10CB8000FBF7B4FD8A20FBF7B1FD0020FBF7AEFDFB
:10CB90000020FBF7ABFD0020FBF7A8FDEDB23878D5
:10CBA000FBF7A4FD2846FBF7A1FD91E7674A507803
:10CBB00093788DF80C303A788DF80D00802103447D
:10CBC0008DF80E100A338A218DF80F1013440021BE
:10CBD00003A88DF810108DF811108DF812108DF833
:10CBE00013208DF81430FCF71BF871E700225B4B23
:10CBF0001A7094F85C30042B04D1554B19780A064E
:10CC000040F1688194F87421082A04D840F2511345
:10CC1000D340DF0701D4FEF767F994F87431092B8C
:10CC20006FD1FBF729FD636A4D4DC01A00282A68B1
:10CC3000B8BF4042904208D94A4B1A78012A04BF33
:10CC400002221A70FBF718FD6062FBF715FDA36A5C
:10CC50006A68C01A0028B8BF4042904208D9414BC8
:10CC60005A78012A04BF02225A70FBF705FDA06220
:10CC7000FBF702FDE36AAA68C01A0028B8BF404269
:10CC8000904208D9374B9A78012A04BF02229A7041
:10CC9000FBF7F2FCE06294F8843093B394F86C31C3
:10CCA0007BBB304A30481D46D15C022940F00681EA
:10CCB00050F823104E1C00F000812C4A84F8683193
:10CCC0001268C4F84C212A4A1268C4F85021226B19
:10CCD000C4F85421274A21631268C4F8582194F8F3
:10CCE0003420C4F85C210023D4F88C20C4F86021DF
:10CCF00084F83430D4F88820C4F86421012384F8FF
:10CD00006C3194F87431092B06D194F85C20022A16
:10CD100004BF052284F85C20D4F87821002A00F0B2
:10CD2000D680092B40F0D38094F85C30012B40F082
:10CD3000CE80216B1048002350F823508D4240F0E4
:10CD4000C280052384F85C30C1E000BF0C80FF1F67
:10CD50007806002034060020280300208F070020DA
:10CD6000F40500204506002008F7FF1F800700207B
:10CD70009C07002080060020F4F7FF1F03A8FBF7A4
:10CD8000CDFC054600284ED0FBF7E0FC08B184F846
:10CD9000A66194F8A6219DF80C10531CDBB2224426
:10CDA000092B84F8A63182F8A7117FF422AF5E4ADE
:10CDB00094F8A71152780023914284F8A6317FF4A9
:10CDC00018AF5A495A5C01331644082BF6B2F9D110
:10CDD00094F8AF31B34222D1554B94F8A8211A7080
:10CDE00094F8A9215A7094F8AA219A7094F8AB216A
:10CDF0009A7194F8AC215A7194F8AD211A7194F893
:10CE0000AE21DA70FBF738FC4A4B4B4A186000231E
:10CE10001370032284F8742184F8A63196E6042363
:10CE200084F87431E5E60AAE3046FBF7E6FE48B317
:10CE30002B46F25C01331544082BEDB2F9D19DF875
:10CE40003020AA42ECD13A4B9DF829201A709DF867
:10CE50002A205A709DF82B209A709DF82C209A71E8
:10CE60009DF82D205A719DF82E201A719DF82F20C3
:10CE7000DA70FBF701FC2F4B18602F4B00221A7061
:10CE8000072361E694F85C30013B012B3FF6B1AE1D
:10CE9000236BB3F5805F0CD2FBF78AFE48B1206BA1
:10CEA0002349431C2363FBF7F1FF092384F8743102
:10CEB00053E6002384F85C309BE6D55401332F2BD6
:10CEC0007FF4F2AE1DE701339A427FF435AF0FB025
:10CED000BDE8F08394F87401082804D840F2511298
:10CEE000C240D207F3D4D4F87001144DD3F8033004
:10CEF0006970B0F5805F6B6012D20D49FBF7B2FF2D
:10CF00000B49D4F87001FCF703F838B1D4F870314C
:10CF10000133C4F8703165232B70D8E70723FBE792
:10CF200007232B7000230DE70C80FF1F1FF8FF1F46
:10CF3000780600203C0600204306002094070020CD
:10CF4000704710B5074CFBF797FB2368C01AB0F584
:10CF5000FA7F05D9044B0222DA60FBF78DFB2060D3
:10CF600010BD00BFA00B002000F00F407047064B23
:10CF70005A7832B9D3F80310044B01B901221A7060
:10CF800070470322024BFAE7780600204F03002087
:10CF9000940700207047704770477047704770478C
:10CFA000024B185C431F58425841704728F8FF1F36
:10CFB00038B505460C46A1B902F00EF9214620F419
:10CFC000E072284602F0E2F860236B431B4AD35C10
:10CFD0009BB328464FF000620721BDE8384002F0BD
:10CFE0003BB9002102F0F8F804F00303022B20F40F
:10CFF000E0721CD0032B1DD0012B01D142F0400266
:10D00000630748BF42F4807214F0080418BF42F46A
:10D0100000720021284602F0B9F8002CD9D1284628
:10D020004FF000620721BDE8384002F023B942F01A
:10D030008002E5E742F0C002E2E738BDC804002004
:10D0400073B5144C23180646DB780D4623B94FF010
:10D05000C052072102F00EF90F4A602303FB06239A
:10D0600001229B7D019285EAE572A2EBE572D2B2C4
:10D07000009206210022304602F05EF8002D04EBFB
:10D08000060304EB8604B4BF01220222DA70A56015
:10D0900002B070BD28F8FF1FC8040020184B1A18F2
:10D0A00073B5D178044641B303EB80030025D570F6
:10D0B00007214FF080529D6002F0CEF84FF00062E1
:10D0C0000721204602F0D6F860230E4A6343D618A3
:10D0D000D35C93B15021204602F07EF82121024614
:10D0E000204602F053F8327DB37D0192727D0092AA
:10D0F00006212A46204602F01FF802B070BD00BF8C
:10D1000028F8FF1FC80400202DE9F347174D2C7D98
:10D1100005F115084CB9E0B2FBF79BFC08F80400D8
:10D120000134082CF7D101232B75DFF848A0104FEC
:10D13000272400264FF00209F0B2FBF78AFC18F80A
:10D14000063083421DD006F1080308F806005AF89D
:10D150002330022B10D0032B02D0012B11D180B130
:10D160003B5D012B08BF07F804900AE028F8FF1F79
:10D1700045060020F405002018B93A5D012A00D1C7
:10D180003B550136082E04F10104D5D1B14CE369B9
:10D19000C3B1B14E3778AFB9FBF76EFAAF4B1B682E
:10D1A000C01A0028E369B8BF404298420AD93846FD
:10D1B00002F0A8F8012002F0A5F8022002F0A2F87F
:10D1C00001233370236AC3B1A54E3778AFB9FBF79B
:10D1D00053FAA44B1B68C01A0028236AB8BF404208
:10D1E00098420AD9384602F08DF8012002F08AF8F8
:10D1F000022002F087F8012333702221687F9A4EC3
:10D2000001F0EAFF4FEA0028687F02F062F80F2180
:10D210000446687F01F0E0FF0746687F642303FB54
:10D2200000631B69002B00F00781002B88EAE8727D
:10D23000A2EBE872B8BF5B429A4240F3FD802B1824
:10D240009B7F43B94FF08062012102F005F86B7FAC
:10D2500001222B449A7704F00903092B31D1687F0E
:10D260008249C21C8B5CDBB2012B0ABF4FF0020E5D
:10D270008B5C01F802E07E490A7818BFB3FA83F3A9
:10D2800042FA00FE18BF5B091EF0010F15D04FF0E7
:10D29000010CDFF800920CFA00FE89F800E0DFF8DC
:10D2A000F89189F800C0DFF8F4C19CF800C0BCF127
:10D2B000000F02D122EA0E020A7013B1092102F016
:10D2C00015F8A10010D5687F684A00F10F03D15C02
:10D2D000012904BF0221D1544FF0005102F006F899
:10D2E0006B7F644A0121D154220507D5B8F1000FA4
:10D2F00004D14FF40061687F01F0F8FFE30407D523
:10D30000B8F1000F04D14FF48051687F01F0EEFFB7
:10D31000A00407D5B8F1000F04D14FF40051687F85
:10D3200001F0E4FF610407D5B8F1000F04D14FF418
:10D330008041687F01F0DAFF687F642303FB0063AC
:10D340001B6A0BB362031FD501F0DCFF5021687F1D
:10D3500001F042FF6B7F484A52F823202121821AB4
:10D36000184601F013FF4FF48021687F01F0BEFFE3
:10D370006B7F3E4903F11502885C012804BF02203F
:10D3800088543E4A0121D1546B7F17F0800105EB90
:10D39000030200F0858092F8211089B9012182F8FA
:10D3A0002110374A1A44127E12F0010F08D00221D0
:10D3B0001B2211FB03232D4AD05C012808BFD15446
:10D3C0006B7FEA1817F4807792F8241074D089B92B
:10D3D000012182F824102A4A1A44D27E12F0010F49
:10D3E00008D00E33214A12F81310012904BF02217C
:10D3F00002F81310FBF740F9AB6AC01A0028B8BF57
:10D4000040420A2840F39680687F1E4B1E4A1F49FF
:10D410001F4F0344024401EB800101F003FE6C7FC7
:10D420002A5D6023052A6BD8DFE812F050008700E0
:10D43000CF00150127016A012B189B7F002B3FF4B9
:10D440000AAF4FF08062012101F014FF6B7F0022D0
:10D450002B44FFE60C80FF1F430600203C06002003
:10D4600028030020340600209803002045060020F1
:10D470006403002090030020580300205003002084
:10D48000F4050020930300204C03002068030020D3
:10D49000C804002056030020740600203803002032
:10D4A00092F8210000288BD082F82110C44A1A4437
:10D4B000127E12F0020F79E700299BD082F82470C7
:10D4C000BF4A1A44D27E12F0020F89E76343FB5C25
:10D4D000B3B1204600F082FE90B91021204601F041
:10D4E000B3FA642303FB046620F4F852737ADB0872
:10D4F00042EA03221021204601F072FA01232B5543
:10D50000687F00F095F96C7F60236343FB5C3BB15F
:10D510002B19DB78012B00F03F81022B00F04881B2
:10D520006B7F0133DBB2022B88BF00236B77FBF7E5
:10D53000A3F8A86202B0BDE8F087002205212046CA
:10D5400001F024FE602202FB04722046117D937DCF
:10D550000191527D00920621002201F0EDFD79211A
:10D56000204601F039FE7F281BDCC0F18006042232
:10D570002021204601F00AFE924A2421204601F093
:10D5800005FE2121204601F027FE37218219204681
:10D5900001F0FCFDFBF770F805EB8403D862022371
:10D5A000ADE7B0F5C07F02DAC0F5C076DFE7B0F5D1
:10D5B000207F02DAC0F52076D9E7B0F5607FB4BFEE
:10D5C000C0F56076C0F59066D1E7FBF755F805EB3E
:10D5D0008403DB6AC01A0028B8BF4042B0F57A7FE6
:10D5E0008EDD642303FB0466F66956B121212046D3
:10D5F00001F0F2FD50210246204601F0C7FD032351
:10D600007DE732462021204601F0C0FD324624212C
:10D61000204601F0BBFD5021204601F0DDFD212117
:10D620000246204601F0B2FD2121204601F0D4FD42
:10D6300037210246204601F0A9FD04222021204680
:10D6400001F0A4FD5F4A2421204601F09FFD5E4BBE
:10D6500001221A55D3E74FF0C0520721204601F0AE
:10D6600009FE5A4A0721204601F0F6FDFBF704F8AF
:10D6700005EB8403D862042341E7FAF7FDFF05EBCD
:10D680008403DB6AC01A0028B8BF4042B0F57A7F35
:10D690007FF736AF4FF019420721204601F0EAFD2F
:10D6A000642303FB0466737E0BB11B0725D54FF083
:10D6B00020620721204601F0CFFD8022052120466F
:10D6C00001F064FD5921204601F086FD602303FB33
:10D6D0000473002218613E4B5021204643F8242059
:10D6E00001F07AFD21210646204601F075FD394BF7
:10D6F000301A43F82400052301E74FF00072D8E701
:10D70000634317F80380B8F1000F7FF4F9AE2046A9
:10D71000FFF7C4FC4FF004620721204601F0AAFD88
:10D7200003220521204601F031FD642303FB04663A
:10D730000621B37DB27A0193737A00932046434663
:10D7400001F0FAFC1021204601F07EF9102140F48E
:10D75000F852204601F044F9F37D05F80480CBB976
:10D7600001222021204601F011FD00222421204623
:10D7700001F00CFD2121204601F02EFD144B53F841
:10D7800024202121821A204601F000FD0E4B0122A7
:10D790001A55B5E60222E4E75021204601F01CFDAF
:10D7A000A0F5C332A03A2121204601F0EFFCB7E6F4
:10D7B0005021204601F010FD00F5C332A032F2E7FF
:10D7C000F405002040420F00530300200000408178
:10D7D0004003002058030020024B03EB80008068C8
:10D7E000704700BF28F8FF1F38B5104A642303FBB9
:10D7F00000230446DB7D0D46B3B90122202101F050
:10D80000C5FC20464FF08052072101F025FD20463F
:10D810004FF00062072101F02DFD2A462046242109
:10D82000BDE8384001F0B2BC0222E7E798030020CF
:10D830002DE9F74F0F210446964D01F0CDFC6422EF
:10D840006243AE18030A317AD6F8049011F0400F03
:10D8500014BFAA5855F802A04FEAD01015BF03F024
:10D86000010800F0010800F0010303F001031CBFF0
:10D87000C2F1000AC9F100090E0601F03F07019349
:10D88000204613D501F04AFEB0FA80FB4FEA5B1B3D
:10D890007A1E019B072A6FD8DFE812F010001000F3
:10D8A00010001000930293029302930201F036FEDF
:10D8B00010F1000B18BF4FF0010BE9E7764E325D17
:10D8C000013A0E2A58D8DFE812F00F0036005A004D
:10D8D00066008900A500C700EF005C01CE01D401FD
:10D8E00057003F02600248024FF064094FF0000801
:10D8F00009FB045A5FFA88F0844208D09AF83E3057
:10D900007BB109FB085292F83E209A4209D10121CD
:10D9100001F062FC614B43F82800614B012208F8DA
:10D92000032008F10108B8F1030FE3D1023F012FF2
:10D930002ED802232DE006EB840301215A682046ED
:10D9400042F0020201F022FC4FF06408002708FBBD
:10D950000459F8B2844208D099F83E3043B108FB2C
:10D96000075292F83E209A4202D15146FFF73CFFFF
:10D970000137032FEDD1375503B0BDE8F08F002BF1
:10D98000FAD02121204601F027FC464B43F8240021
:10D9900004233355F0E706EB840301215A6820463F
:10D9A00042F0010201F0F2FB4FF06408002708FB8F
:10D9B0000459F8B2844208D099F83E304BB108FBC4
:10D9C000075292F83E209A4203D1CAF10001FFF7B4
:10D9D0000BFF0137032FECD10523DAE7B8F1000F75
:10D9E000CAD04FF06408002708FB0459FBB2A342D9
:10D9F00008D099F83E3043B108FB075292F83E2018
:10DA00009A4202D1384601F07DFC0137032FEDD157
:10DA10000623BEE706EB840301215A68204622F064
:10DA2000030201F0B3FB4FF06408002708FB045A1F
:10DA3000F8B2844208D09AF83E3043B108FB07524E
:10DA400092F83E209A4202D14946FFF7CDFE0137B7
:10DA5000032FEDD107239CE7B8F1000F8CD1642789
:10DA600007FB045A5FFA88F0844208D09AF83E30E7
:10DA70004BB107FB085292F83E209A4203D1C9F1FC
:10DA80000001FFF7B1FE08F10108B8F1030FE9D179
:10DA900008237EE79803002060F8FF1F64F8FF1F4B
:10DAA000530300202C030020B8F1000F3FF464AFB3
:10DAB0002121204601F090FB4FF0640882460027A8
:10DAC00008FB045BF8B2844208D09BF83E3043B1B7
:10DAD00008FB075292F83E209A4202D10021FFF73C
:10DAE00083FE0137032FEDD1C94A52F82430A3EB4E
:10DAF0000A0342F8243006EB840301215A682046C9
:10DB000022F003024FF0640801F040FB08FB0453CD
:10DB10004FF0000B01935FFA8BF7BC4209D0019BD9
:10DB200093F83E2022B308FB0B5191F83E1091422E
:10DB30001ED108FB0B52D27D0ABB0522202138469C
:10DB400001F024FB4A462421384601F01FFB4FF028
:10DB500080520721384601F08DFB4FF0006207210B
:10DB6000384601F079FB52463721384601F00EFB6A
:10DB70000BF1010BBBF1030FCDD1092309E70622FD
:10DB8000DCE70F21204601F027FBC1077FF5F4AE4B
:10DB90002121204601F020FB9E4B4FF0640A43F800
:10DBA00024004FF000080AFB045B5FFA88F084420F
:10DBB00008D09BF83E3043B10AFB085292F83E2051
:10DBC0009A4202D10021FFF70FFE08F10108B8F1D7
:10DBD000030FEAD14FF0640B4FF000080BFB045326
:10DBE0005FFA88FA544508D093F83E20C2B10BFB87
:10DBF000085191F83E10914212D10022372150462F
:10DC0000019301F0C3FA00222121504601F0BEFA2F
:10DC10005021504601F0E0FA7F4A019B42F828006B
:10DC200008F10108B8F1030FDAD1033F012F00F228
:10DC300092804FF06408002708FB045AF8B284422F
:10DC400008D09AF83E304BB108FB075292F83E20BC
:10DC50009A4203D1C9F10001FFF7C6FD0137032F36
:10DC6000ECD10A2395E6B8F1000F3FF485AE0B2303
:10DC70008FE6B8F1000F7FF47FAE2121204601F03E
:10DC8000ABFA6427824607FB045B5FFA88F08442A4
:10DC900008D09BF83E3043B107FB085292F83E2073
:10DCA0009A4202D10021FFF79FFD08F10108B8F167
:10DCB000030FEAD14FF002089AFBF8F84FF0640A1C
:10DCC0000AFB04534FF0000B01935FFA8BF7BC4241
:10DCD00009D0019B93F83E206AB30AFB0B5191F8DF
:10DCE0003E10914227D14D4A52F82B20012122F0BB
:10DCF0000302384601F04AFA0AFB0B52D27D0ABBF6
:10DD000005222021384601F041FA4A4624213846AE
:10DD100001F03CFA4FF080520721384601F0AAFA90
:10DD20004FF000620721384601F096FA424637214B
:10DD3000384601F02BFA0BF1010BBBF1030FC4D1F4
:10DD40000D2326E60622DCE70F21204601F044FAE7
:10DD5000C2077FF511AE0E231BE64FF064080027C3
:10DD600008FB0459F8B2844208D099F83E3043B118
:10DD700008FB075292F83E209A4202D10021FFF799
:10DD800033FD0137032FEDD1E5E74FF0640800279D
:10DD900008FB0459F8B2844208D099F83E305BB1D0
:10DDA00008FB075292F83E209A4205D11B4B0121F5
:10DDB00053F8272001F0EAF90137032FEAD10023B5
:10DDC000E7E5174E325D013A0E2A3FF6D5AD01A1C7
:10DDD00051F822F025DE000075DE0000CFDE0000E5
:10DDE000EDDE000049DF000079D9000065DF0000AA
:10DDF00079D9000079D900000FE0000027E0000089
:10DE0000B9DF0000CBE0000081E100003FE100004D
:10DE10002C030020E80500205803002064F8FF1FB1
:10DE200060F8FF1F4FF064094FF0000809FB045A27
:10DE30005FFA88F0844208D09AF83E3073B109FB4B
:10DE4000085292F83E209A4208D1C94B012108F8A5
:10DE5000031001F0C1F9C74B43F8280008F101088D
:10DE6000B8F1030FE4D1062F3FF463AD082F7FF420
:10DE70008FAD5EE5062F22D106EB84035A6822F0AF
:10DE8000030242F002020121204601F07FF94FF027
:10DE90006408002708FB0459F8B2844208D099F8B6
:10DEA0003E3043B108FB075292F83E209A4202D11D
:10DEB0005146FFF799FC0137032FEDD15BE5082FA1
:10DEC000E5D106EB84035A6822F00302DBE77A1FF0
:10DED000012A05D823B1062F3FF45AAD0F2358E588
:10DEE000BBF1000F3FF448AD0C2352E5052F23D1C1
:10DEF00006EB84035A6822F0030242F0010201217A
:10DF0000204601F043F94FF06408002708FB04594C
:10DF1000F8B2844208D099F83E304BB108FB075262
:10DF200092F83E209A4203D1CAF10001FFF75CFC4F
:10DF30000137032FECD14FE5072FE4D106EB840323
:10DF40005A6822F00302DAE77B1F012B05D8B8F1EB
:10DF5000000F02D0052FC1D1EBE4BBF1000F3FF45D
:10DF60000BAD77E5BBF1000F7FF406AD073F012F46
:10DF70000AD906EB840301215A6822F0030242F019
:10DF80000202204601F002F94FF06408002708FB66
:10DF9000045AF8B2844208D09AF83E3043B108FBE4
:10DFA000075292F83E209A4202D14946FFF71CFCE4
:10DFB0000137032FEDD154E6BBF1000F7FF4DCAC49
:10DFC000073F012F0AD906EB840301215A6822F08A
:10DFD000030242F00102204601F0D8F84FF0640835
:10DFE000002708FB045AF8B2844208D09AF83E3061
:10DFF0004BB108FB075292F83E209A4203D1C9F177
:10E000000001FFF7F1FB0137032FECD129E6BBF14B
:10E01000000F3FF4B1AC2121204601F0DDF806EB02
:10E020008403186123E6BBF1000F7FF4A5AC212126
:10E03000204601F0D1F84FF0640808FB04538246F3
:10E0400001935FFA8BF7BC4209D0019B93F83E2005
:10E050009AB308FB0B5191F83E1091422DD1454ADD
:10E0600052F82B20012122F00302384601F08EF8ED
:10E0700008FB0B52D27D32BB05222021384601F02D
:10E0800085F84A462421384601F080F84FF0805246
:10E090000721384601F0EEF84FF0006207213846BC
:10E0A00001F0DAF806EB8402022112693846524484
:10E0B00092FBF1F2372101F069F80BF1010BBBF192
:10E0C000030FBED13CE60622D7E70F21204601F020
:10E0D00083F8C3077FF550AC0E232121204633552A
:10E0E00001F07AF8244B4FF0640843F8240000262E
:10E0F00008FB0459F7B2BC4208D099F83E30D3B1BE
:10E1000008FB065292F83E209A4214D1002138466C
:10E11000FFF76AFB00223721384601F037F800226A
:10E120002121384601F032F85021384601F054F8E8
:10E13000124B43F826000136032EDBD11CE44FF0CE
:10E140006408002708FB0459F8B2844208D099F803
:10E150003E3043B108FB075292F83E209A4202D16A
:10E160000021FFF741FB0137032FEDD1F3E500BF9D
:10E170005303002064F8FF1FE80500205803002027
:10E180004FF06408002708FB0459F8B2844208D015
:10E1900099F83E305BB108FB075292F83E209A4254
:10E1A00005D1054B012153F8272000F0EFFF01377F
:10E1B000032FEAD103E600BF64F8FF1F024B1A5C8D
:10E1C0000AB901221A54704760F8FF1F024B1A5C0B
:10E1D0000AB10F221A54704760F8FF1F014B185CF8
:10E1E000704700BF60F8FF1F0C4A116940F27323AB
:10E1F0004B434FF6FF71B3FBF1F36E2B06D9084B7F
:10E200004FF4802159605723136070474F2B9EBFF6
:10E21000034B4FF480219960F5E700BF00B0034045
:10E2200080F00F401B4B1A6802F01F02072A2ED8FD
:10E23000DFE802F0040B2D11171D23291A69164976
:10E2400092B20A8041221A6070471A69124992B24A
:10E250004A804322F7E71A690F4992B2CA804422E2
:10E26000F1E71A690C4992B20A814522EBE71A6973
:10E27000094992B24A814622E5E71A69064992B2F3
:10E280008A814722DFE71A69034992B2CA81402294
:10E29000D9E700BF00B00B407CF8FF1F38B541F252
:10E2A0003001114B5A5842F000625A5041F23C0181
:10E2B00000245A5842F000625A5003F5E8230C2516
:10E2C00040229D604920DC605C621A6001F054F9D4
:10E2D000064B57229D602720DC605C621A60BDE817
:10E2E000384001F049B900BF0070044000B003405D
:10E2F0000B2829D8DFE800F0060A0D102828282866
:10E3000013281E23114B188980B270470F4B588970
:10E31000FAE70E4B9889F7E70C4BD889F4E70B4BDB
:10E32000588883B240F2732058434FF6FF7390FB36
:10E33000F3F07047054BD88883B28E20F4E7034B87
:10E34000188883B24220EFE7002070477CF8FF1F57
:10E3500030B52E4D41F23C042B5943F010032B51A4
:10E360002B4B4FF400741C636FF4F8755C63A3F5DA
:10E370001433A4F13E542C441C604FF400545C60F0
:10E38000244C1C601C68E401FCD50138072834D8F3
:10E39000DFE800F0312F2D2B293327041E48586069
:10E3A0001E4B002058631E4818601E484FF08064C2
:10E3B00000EA8145C3F88040C3F88450FAB100EA0E
:10E3C0008240C3F89040C3F894004FF08460C3F8D3
:10E3D000A000C3F8A410AAB1C3F8B000C3F8B420D9
:10E3E00030BD1148DBE71148D9E71148D7E711489C
:10E3F000D5E71148D3E71148D1E71148CFE7C3F873
:10E400009020E2E7C3F8B02030BD00BF00700440A8
:10E41000009004400F0080508720FE010040024021
:10E420000F0080000000FC1F8720FE038720FE0FE6
:10E430008720FE138720FE278720FE638720FEC7E4
:10E440008720FE07384AD2F88030C3F30363022BDB
:10E450005FD0D2F89030C3F30363022B5BD0D2F8C5
:10E46000A030C3F30363022B06D0D2F8B030C3F35D
:10E470000363022B56D103231B0103F1402202F553
:10E480000032D2F88010C1F303410170D2F880103D
:10E4900011F4801118BF01218170D2F8801011F49D
:10E4A000001118BF012141704178B1BBD2F884102E
:10E4B000C1F38A4103F1402303F500334160D3F8EF
:10E4C0008810090E0172D3F88810090C4172D3F834
:10E4D0008810090A8172D3F88810C172D3F88C10A1
:10E4E000090E0173D3F88C10090C4173D3F88C100A
:10E4F000090A8173D3F88C30C373D2F880309B0241
:10E500004CBF4FF084634FF08063C2F8803001202D
:10E5100070470023B0E70123AEE7D2F8841021F062
:10E520006041C7E70020704700400240184AD2F817
:10E530007031C3F303630C2B10B527D044784368C4
:10E5400004B3C3F31103C2F874318368104A1BBAD1
:10E55000C2F87831C3681BBAC2F87C318378002CCA
:10E5600014BF4FF042624FF040620BB142F4801290
:10E5700003781B0403F470231343054A0120C2F8F7
:10E58000703110BD034901EA8343DCE7002010BD70
:10E59000004002400000FC1F0B4B4FF00062C3F82C
:10E5A00070214FF48022C3F87421084AC3F87821FF
:10E5B0006FF48471A2F166320A44C3F87C21044AE4
:10E5C000C3F87021704700BF0040024078563412F3
:10E5D0000000080C10B53A4BDA7842F00202DA700B
:10E5E000384A1078C0B20228114641D0032835D0ED
:10E5F000012832D1546891688C4215D2D978C90764
:10E6000007D45168D0684C1C5460425CD2B21A7175
:10E6100010BD997801F0DF019970997801F0EF0150
:10E6200099701074002317E0517C01F0FF0049B984
:10E63000997801F0DF019970997801F0EF019970F4
:10E64000107010BD997841F004019970917CC9B2A5
:10E650001971002353740323137010BD997801F0CE
:10E66000EF0199701B795169DBB20B700223F3E75C
:10E670009469D06984421DD2D2698869121A012A2C
:10E6800005D19A7802F0DF029A7000230B70CB69F3
:10E690008A699B1A022B9FBF094A937843F00803AB
:10E6A00093708A694869531C8B61054B1B79DBB2F7
:10E6B000835410BD997801F0DF019970B2E700BF73
:10E6C0000070064090F8FF1F41F234020A498B584F
:10E6D00043F080038B50094B4FF418729A62DA6250
:10E6E00003F5E0331B225A70C0229A7000225A713F
:10E6F000192000F041BF00BF0070044000B004408A
:10E7000010B5104B00241C745C749A6001225C608C
:10E710001A700D4AD960917801F0F70191709178E3
:10E7200041F010019170917800F0FE0041F020015D
:10E73000917010711A78002AFCD1187CB0FA80F020
:10E74000400910BD90F8FF1F0070064010B5104B37
:10E7500000241C745C74DA6103229C611A700D4AF7
:10E760005961917801F0F7019170917841F01001B1
:10E770009170917840F0010041F02001917010718A
:10E780001A78002AFCD1187CB0FA80F0400910BD3C
:10E7900090F8FF1F0070064070B5144C00256361AF
:10E7A0000126049B25746674A2606560E36140EAFB
:10E7B0000603A561A3740E4BE16026709A7802F0FF
:10E7C000F7029A709A7842F010029A709A7800F0E4
:10E7D000FE0042F020029A7018712378002BFCD1C1
:10E7E000207CB0FA80F0400970BD00BF90F8FF1F98
:10E7F000007006402DE9F3411B4F1C4C00264FF0E2
:10E800000C08F5B20423BA8FCDF800800A212846FF
:10E8100000F03EFD4FF480520021284600F0B6FC87
:10E82000FA695421284600F0B1FC00225021284604
:10E8300000F0ACFC626CFF21082384F8401084F8DF
:10E840004130019100936321D3B22846C2F30722DD
:10E85000013600F071FC032E07F1640704F1600437
:10E86000CFD102B0BDE8F08198030020C804002099
:10E8700038B50D460721044600F0AEFCEB074CBF4F
:10E8800040F0800220F08002A8074CBF42F4807262
:10E8900022F4807269074CBF42F0100222F010028D
:10E8A0002B074CBF42F4007222F40072E8064CBF02
:10E8B00042F0040222F00402A9064CBF42F0080212
:10E8C00022F008026B064CBF42F0200222F0200228
:10E8D00028064CBF42F0400222F04002E9054CBF3E
:10E8E00042F0020222F00202AB0520464CBF42F485
:10E8F000806222F480620721BDE8384000F046BC07
:10E90000072108B500F068FCC0F3C013C20548BF7A
:10E9100043F00203C10648BF43F00403820548BF29
:10E9200043F00803410748BF43F01003020748BF04
:10E9300043F02003810648BF43F04003420648BF2E
:10E9400043F08003810748BF43F48073420548BF0A
:10E9500043F40073184608BD2DE9F74305460C46FD
:10E9600091460C216FF0007298469DF828709DF832
:10E970002C6000F00BFC0E21284600F02DFC4FF01F
:10E98000FF320C21284600F001FC44F08003019383
:10E9900000231A4600936D21284600F0CDFB019616
:10E9A000009743464A466C21284600F0C5FB0E21DD
:10E9B000284600F011FC8301F9D504F07F0448EAF1
:10E9C000092804EB440447EA08272C44034B46EA91
:10E9D000072643F8246003B0BDE8F083B0F8FF1FBA
:10E9E00073B505460C4616460C216FF0007200F018
:10E9F000CDFB0E21284600F0EFFB4FF0FF320C213B
:10EA0000284600F0C3FB44F08003019300231A461C
:10EA10006D212846009300F08FFB32466C2128467A
:10EA200000F0B4FB0E21284600F0D6FB8301F9D597
:10EA300004F07F0404EB44042C44024B43F82460AC
:10EA400002B070BDB0F8FF1F73B51F4B01F07F041B
:10EA500005461B5D83B36FF000720C2100F096FB3E
:10EA60000E21284600F0B8FB00264FF0FF320C21A3
:10EA7000284600F08BFB32466D2128460194009613
:10EA8000334600F059FB32466C21284600F07EFBED
:10EA90000E21284600F0A0FB8201F9D56E21284600
:10EAA00000F09AFB222C01D0422C03D1030201D5A5
:10EAB00040F07F4002B070BD04EB44040444034BBB
:10EAC00053F82400F6E700BF84210100B0F8FF1FCF
:10EAD00070B50B4C2218054692F800260E465AB91E
:10EAE0006C21FFF7B1FF06F00F0320F00F021A436D
:10EAF0006C212846FFF774FF631983F8036670BD25
:10EB0000B0F8FF1F38B50C466C210546FFF79CFF97
:10EB1000240104F0700420F07002224328466C2186
:10EB2000BDE83840FFF75CBF38B50C466C210546A0
:10EB3000FFF78AFFE40304F4C03420F4C032224318
:10EB400028466C21BDE83840FFF74ABF38B50C466F
:10EB50006C210546FFF778FF240504F4700420F4C7
:10EB60007002224328466C21BDE83840FFF738BFC9
:10EB700038B50C466C210546FFF766FF240604F005
:10EB8000706420F07062224328466C21BDE8384052
:10EB9000FFF726BF38B50D466C210446FFF754FF3A
:10EBA0003DB140F0804220466C21BDE83840FFF77F
:10EBB00017BF20F08042F6E738B50D466C210446B9
:10EBC000FFF742FF3DB140F4002220466C21BDE832
:10EBD0003840FFF705BF20F40022F6E738B50D46B0
:10EBE0006C210446FFF730FF3DB140F480222046FF
:10EBF0006C21BDE83840FFF7F3BE20F48022F6E731
:10EC000038B50D466C210446FFF71EFF3DB140F4B8
:10EC1000804220466C21BDE83840FFF7E1BE20F479
:10EC20008042F6E738B50D466C210446FFF70CFF2D
:10EC30003DB140F4005220466C21BDE83840FFF75A
:10EC4000CFBE20F40052F6E738B50D466C210446DD
:10EC5000FFF7FAFE3DB140F4805220466C21BDE83A
:10EC60003840FFF7BDBE20F48052F6E738B50C46B9
:10EC70006C210546FFF7E8FE230748BF20F070002F
:10EC80004FEA04124CBF40F4006020F4076002F029
:10EC9000700202436C212846BDE83840FFF7A0BE51
:10ECA00038B50C466C210546FFF7CEFEE40104F4AE
:10ECB000F06420F4F062224328466C21BDE838401D
:10ECC000FFF78EBEFFF7ECBF08B5074B034493F880
:10ECD00000262AB96C21FFF7B7FE00F00F0008BD2F
:10ECE00093F8030608BD00BFB0F8FF1F08B56C21FC
:10ECF000FFF7AAFEC0F3021008BD08B56C21FFF7AC
:10ED0000A3FEC0F3C13008BD08B56C21FFF79CFE1F
:10ED1000C0F3035008BD08B56C21FFF795FEC0F3A2
:10ED2000036008BD08B56C21FFF78EFEC0F380704C
:10ED300008BD08B56C21FFF787FEC0F3C04008BDD1
:10ED400008B56C21FFF780FEC0F3804008BD08B510
:10ED50006C21FFF779FEC0F3803008BD08B56C2147
:10ED6000FFF772FEC0F3403008BD08B56C21FFF715
:10ED70006BFEC0F3003008BD08B56C21FFF764FEE0
:10ED8000C0F30213020548BF43F00803184608BD4C
:10ED900008B56C21FFF758FEC0F3C31008BDFFF79C
:10EDA000F7BF38B50C466D210546FFF74DFE6401EF
:10EDB00004F0600420F06002224328466D21BDE883
:10EDC0003840FFF70DBE38B50C466D210546FFF7FC
:10EDD0003BFE640304F4C04420F4C04222432846AE
:10EDE0006D21BDE83840FFF7FBBD38B50C466D21FD
:10EDF0000546FFF729FE240204F4706420F47062D3
:10EE0000224328466D21BDE83840FFF7E9BD38B5FB
:10EE10000C466D210546FFF717FE04F00F0420F0A5
:10EE20000F02224328466D21BDE83840FFF7D8BDC8
:10EE300038B50D466D210446FFF706FE20F47F002D
:10EE400040EA05426D212046BDE83840FFF7C8BDC5
:10EE500038B50D466D210446FFF7F6FD3DB140F48F
:10EE6000004220466D21BDE83840FFF7B9BD20F4CF
:10EE70000042F6E738B50D466D210446FFF7E4FD84
:10EE80003DB140F0807220466D21BDE83840FFF76B
:10EE9000A7BD20F08072F6E708B56D21FFF7D4FD1D
:10EEA000C0F3411008BD08B56D21FFF7CDFDC0F3DB
:10EEB000413008BD08B56D21FFF7C6FDC0F3032042
:10EEC00008BD08B56D21FFF7BFFD00F00F0008BDBC
:10EED00008B56D21FFF7B8FD0314D8B21B0648BF73
:10EEE00060F0FF0008BD08B56D21FFF7ADFDC0F370
:10EEF000C03008BD08B56D21FFF7A6FDC0F3006066
:10EF000008BD38B50C4670210546FFF79DFD04F09D
:10EF1000030420F4401242EA045228467021BDE85E
:10EF20003840FFF75DBD38B50D4670210446FFF748
:10EF30008BFD3DB140F4002220467021BDE83840F1
:10EF4000FFF74EBD20F40022F6E738B50D467021DC
:10EF50000446FFF779FD3DB140F480222046702140
:10EF6000BDE83840FFF73CBD20F48022F6E738B515
:10EF70000C4670210546FFF767FD04F0030420F4FA
:10EF8000403242EA044228467021BDE83840FFF78B
:10EF900027BD38B50D4670210446FFF755FD20F416
:10EFA0007F4040EA052270212046BDE83840FFF747
:10EFB00017BD38B50D4670210446FFF745FD20F01A
:10EFC000FF0045EA000270212046BDE83840FFF707
:10EFD00007BD08B57021FFF737FDC0F3015008BD2C
:10EFE00008B57021FFF730FDC0F3C04008BD08B57B
:10EFF0007021FFF729FDC0F3804008BD08B57021DE
:10F00000FFF722FDC0F3014008BD08B57021FFF7EE
:10F010001BFDC0F3072008BD08B57021FFF714FDE4
:10F02000C0B208BD70B50E466C2115461C4600F0F6
:10F03000D3F816B1C0F30903336015B1C0F304432C
:10F040002B700CB1000E207070BD2DE9F341F9F763
:10F0500013FB0446F9F710FB001B0028B8BF404221
:10F060000928F7DD0024DFF888801F4F2646E5B227
:10F070004FF0011200212846FFF7B2FC0222532371
:10F080008DE80C006C21412300222846FFF764FC28
:10F09000032106238DE80A0000231A460921284689
:10F0A000FFF75AFC0A21019101230022284600960D
:10F0B000FFF752FC1F230193009300231A461021EF
:10F0C0002846FFF749FC424670212846FFF788FC96
:10F0D0002846FFF7F9FD054B3855E6540134032C5B
:10F0E000C5D102B0BDE8F081B3FEFF1FB0FEFF1F27
:10F0F0001E000CC438B5074C044494F8001641B9FE
:10F1000094F80356FFF7E4FC012384F8003684F8F2
:10F11000035638BDB0F8FF1F064B034493F8002692
:10F1200032B1002293F8031683F80026FFF7D0BC13
:10F13000704700BFB0F8FF1F2DE9F0411F46124B8A
:10F140009DF8186033F810409DF81C50904641F02F
:10F15000800100222046F9F7BBFD414600222046EF
:10F16000F9F7B6FD394600222046F9F7B1FD3146E0
:10F1700000222046F9F7ACFD294620460122BDE8D1
:10F18000F041F9F7A5BD00BF4C80FF1F38B5114B0A
:10F1900033F81040154641F0800100222046F9F76F
:10F1A00097FD290E00222046F9F792FDC5F307418D
:10F1B00000222046F9F78CFDC5F3072100222046E6
:10F1C000F9F786FDE9B220460122BDE83840F9F79B
:10F1D0007FBD00BF4C80FF1F38B51E4B33F8104079
:10F1E000002220460D46F9F773FD00221146204605
:10F1F000F9F76EFD002211462046F9F769FD00225D
:10F2000011462046F9F764FD012200212046F9F756
:10F210005FFD294600222046F9F75AFD00221146DB
:10F220002046F9F755FD0022114605022046F9F760
:10F230004FFD0022114605432046F9F749FD2D02F6
:10F240000543012200212046F9F742FD2D02284303
:10F2500038BD00BF4C80FF1F70B504460D461646F2
:10F26000FFF7BAFF294640EA06022046BDE8704093
:10F27000FFF78CBF70B504460D461646FFF7ACFF8E
:10F28000294620EA06022046BDE87040FFF77EBF0F
:10F290002DE9F8439DF8209098460F4606461446FF
:10F2A0000025FFF799FFC1444146012349450BD38F
:10F2B00004FA08F444402C4080EA040239463046FF
:10F2C000BDE8F843FFF762BF03FA01F215430131CD
:10F2D000ECE710B50C2104464FF0FF32FFF756FF64
:10F2E00020460E21BDE81040FFF776BF10B5CA4397
:10F2F00004460C21FFF74AFF20460E21BDE81040CE
:10F30000FFF76ABF10B5084BC4B201221A5420217E
:10F3100020460022FFF73AFF204600222421BDE8C4
:10F320001040FFF733BF00BF530300202DE9F74320
:10F330000027714E714DDFF8CC91B846FCB24FF406
:10F34000805200212046FFF721FF4FF005121021C7
:10F350002046FFF71BFF4A4604212046FFF716FF11
:10F360006FF000720C212046FFF710FF0E2120469F
:10F37000FFF732FF00231A466D212046CDF80480A6
:10F38000CDF80080FFF7D8FE00226C212046FFF761
:10F39000FDFE032205212046FFF7F8FE042220216E
:10F3A0002046FFF7F3FE002237212046FFF7EEFE4E
:10F3B000002221212046FFF7E9FE4FF448022421D4
:10F3C0002046FFF7E3FE4FF4483228212046FFF79E
:10F3D000DDFE4FF4483229212046FFF7D7FEB37DEA
:10F3E0000193737AB27A0093062100232046FFF737
:10F3F000A3FEB38A424A15215A432046FFF7C6FEB0
:10F400006A6860212046FFF7C1FEAA686121204694
:10F41000FFF7BCFEEB892A7B1C2143EA024220460F
:10F42000FFF7B4FE2A6959212046FFF7AFFE2A6A8A
:10F430005A212046FFF7AAFE6A6A5B212046FFF7A1
:10F44000A5FEAA6A95F82C30D1B2C2F30722019129
:10F4500000925D2100222046FFF76EFE2A6B5E219E
:10F460002046FFF793FEAA6918212046FFF78EFE7B
:10F47000EA6919212046FFF789FE6A6B5C21204664
:10F48000FFF784FEAA6B5F212046FFF77FFEEA6B41
:10F4900052212046FFF77AFE6A6C95F840300193BE
:10F4A00095F8413000936321D3B22046C2F307227E
:10F4B000FFF742FE95F84830CDF8048000227D2108
:10F4C0002046CDF80080FFF737FE4FF4403201218F
:10F4D0002046FFF75BFE01376FF0004235212046E2
:10F4E000FFF754FE032F06F1640605F160057FF473
:10F4F00025AF03B0BDE8F08398030020C8040020C6
:10F50000007102008D124084034B10229A6000BFEC
:10F5100000BF00BF5A60704700F00F4008B50F21D0
:10F52000FFF75AFEC0F3003008BD000270478000AC
:10F53000704700127047801070477047FEE74FF029
:10F54000E0210B4A0B4BC1F8083D4CF22053D3810C
:10F550004DF62813D381138823F001031B041B0CE1
:10F560001380D1F8883D43F47003C1F8883D70479B
:10F570000020054000800000802800F01F014FF0AF
:10F5800001030F4A04DD8B40C2F88C31D360704711
:10F59000402804DD8B40C2F88831936070472028F2
:10F5A00004DD8B40C2F8843153607047404200F064
:10F5B0001F0058BF41428B40C2F880311360704732
:10F5C00000E100E0802800F01F024FF001030D4928
:10F5D00003DD9340C1F88C307047402803DD934031
:10F5E000C1F888307047202803DD9340C1F884308B
:10F5F0007047404200F01F0058BF42429340C1F89C
:10F600008030704700E100E0074B1A78D2B2012A3F
:10F6100002D1222903D15A7001225A707047212940
:10F62000FAD10022F7E700BFB6FEFF1F70B51546FE
:10F6300011B91B4B197070BD022903D1184B01225F
:10F640001A7070BD04291AD1154B5B78012B25D196
:10F650009488402C28BF402400235E1CDBB2A342C8
:10F6600007D300231A4602211846BDE8704000F077
:10F6700047BF2A68D05C00F0C3F83346EDE70329A2
:10F6800006D1074A5378012B08D100239370E9E78C
:10F69000052901BF024B00221A705A7070BD00BFCD
:10F6A000B6FEFF1F10B50446204600F0C1F8002842
:10F6B000FAD110BD704738B50A4C012502460B46F9
:10F6C00000202946A57000F0F5FA224618B1002363
:10F6D000A370122038BD937803F0FF00002BFAD1FD
:10F6E00038BD00BFB6FEFF1FF8B506460F4600F056
:10F6F000F4FC0E4B1A78012A16D15B78012B13D13A
:10F7000000F000F988B10025ECB2A74205D82146E7
:10F710003046BDE8F840FFF7CEBF301900F0D6F80C
:10F7200001350028F0D0F2E70C20F8BDB6FEFF1F2F
:10F7300008B540210248FFF7D7FF00F095F808BD53
:10F74000B9FEFF1F38B5054600F0A8F80B2804469F
:10F7500009D140210548FFF7C7FF28B92846BDE871
:10F76000384000F09BB80024204638BDF9FEFF1F4A
:10F7700070B50C46461E00250CB9284670BD16F81B
:10F78000010FFFF7DFFF013C002818BF0B25A4B2D3
:10F79000F2E738B5451E002415F8010F08B92046D8
:10F7A00038BDFFF7CFFF002818BF0B24F4E707B5DB
:10F7B0000123002200930649064B104600F020FA70
:10F7C000002814BF1B20002003B05DF804FB00BF1D
:10F7D0002DF6000009F6000038B50C46054600F08D
:10F7E00097F8A0420AD32C440020A54207D000B1CC
:10F7F00038BD15F8010B00F051F8F6E70B2038BDC5
:10F8000010B50A4A117840290ED05378D418013324
:10F81000DBB2402BA07001F101014FF0000011702C
:10F8200014BF5370507010BD0B2010BD39FFFF1F67
:10F8300010B50C4A117891B192F84230D4180133C6
:10F84000DBB2A4780470402B4FF0000001F1FF31CF
:10F85000117014BF82F8423082F8420010BD0A20B5
:10F8600010BD00BF39FFFF1F014B1878704700BF64
:10F8700039FFFF1F024B1878C0F14000C0B270473B
:10F8800039FFFF1F034B00225A7083F842201A7081
:10F89000704700BF39FFFF1FFFF7F4BF10B50A4ADA
:10F8A000117840290ED05378D4180133DBB2402BA5
:10F8B000A07001F101014FF00000117014BF5370EE
:10F8C000507010BD0B2010BD7CFFFF1F10B50C4AFF
:10F8D000117891B192F84230D4180133DBB2A47898
:10F8E0000470402B4FF0000001F1FF31117014BF84
:10F8F00082F8423082F8420010BD0A2010BD00BFDD
:10F900007CFFFF1F014B1878704700BF7CFFFF1F73
:10F91000024B1878C0F14000C0B270477CFFFF1F57
:10F92000034B00225A7083F842201A70704700BFC0
:10F930007CFFFF1FFFF7F4BF70B50546007801F0AC
:10F9400093F902780023D9B2914207D25C1C03EBF1
:10F95000830303445E786B789E4227D1174C2B7A41
:10F96000342202FB0142D67813B334234B43E2180E
:10F97000907886420CD000F0030204330C2010FB78
:10F9800002302118205C0B894A68497800F090FB0E
:10F99000D4F89C3083B12A46287812F8081F002931
:10F9A0000CBF03210521BDE8704018472346CAE774
:10F9B000937801339370D8E770BD00BFC0FFFF1F7D
:10F9C0002DE9F04F85B00D4690468DF80F0001F0FF
:10F9D0004BF9022D064647D1077800235C1CDBB2A9
:10F9E000BB4210DB4FF00009DFF8B0B0CA465FFA47
:10F9F00089F4A74212DC284BD3F89C30002B45D168
:10FA000005B0BDE8F08F03EB830333440DF10F0025
:10FA1000DA78597801F0E2F92346DFE704EB840451
:10FA20003444E378A2886178CDF804A0A0780090EF
:10FA30000DF10F0001F0B0F9A378032B05D15A4660
:10FA400061789DF80F0001F031FA6178E37841F0B8
:10FA5000100141EAC3110022C9B20DF10F0001F0FB
:10FA6000EDF909F10109C2E7002DC4D10A49037873
:10FA7000342000FB03138A1C3633294634329A4261
:10FA8000B9D002F8341C02F8331CF7E74246294685
:10FA90009DF80F009847B3E7C0FFFF1F39F900003A
:10FAA000F0B40C7804F06004202C1D4632D14C7860
:10FAB000042C1DD00AD8012C04D003D3022C20D052
:10FAC000032C12D000202880F0BC7047212C1BD0C2
:10FAD00004D8202CF6D1F0BC00F040B9222C16D06E
:10FAE000232CEFD1F0BC00F049B9F0BC00F049B9CB
:10FAF00002241C801468002525701468671C176098
:10FB00006570F0BC00F056B9F0BC00F01FB9F0BC55
:10FB100000F076B9402C06D1044CD4F8A04014B1C2
:10FB2000A446F0BC6047CD20CEE700BFC0FFFF1F5A
:10FB300073B50446007801F097F863680093A27AE1
:10FB4000637A43EA0223ADF8043002780023D9B285
:10FB5000914207D25D1C03EB830303445E78637814
:10FB60009E4225D1174D237A342202FB0152D678CA
:10FB700003B334234B43EA18907886420CD000F04C
:10FB8000030204330C2010FB02302918285C0B8977
:10FB90004A68497800F08CFAD5F89C3033B1227A63
:10FBA00020785AB104F108020521984702B070BDCF
:10FBB0002B46CCE7937801339370DAE76A4603214A
:10FBC000F3E700BFC0FFFF1F07B543680093437A08
:10FBD000817A43EA0123ADF80430084BD3F89C3016
:10FBE00002462BB1017A007829B1083205219847E5
:10FBF00003B05DF804FB6A460421F8E7C0FFFF1F6D
:10FC00002DE9F84305460F461646984601F02CF8B4
:10FC100002789DF8203001328146D2B20021284678
:10FC200001F09EF80446E8B9164A1749284600F044
:10FC300086F999F80000154B342200FB022209F1E5
:10FC400001011A4499463433934201F105010CD164
:10FC50004146284600F074F8044618B9C9F89C706B
:10FC6000C9F8A0602046BDE8F88311F8050C03F838
:10FC7000340C11F8040C03F8330C03F8324C03F87D
:10FC8000314CE0E7A1FA0000C1F90000C0FFFF1FFE
:10FC900008B5074B0022C3F89C20C3F8A02000F051
:10FCA000A1F918B9BDE8084001F06EB808BD00BF61
:10FCB000C0FFFF1F2DE9F041984605460E46174646
:10FCC00000F0D2FF04780023D9B2A14207D2013359
:10FCD00003EB8302024412F8042CB242F4D1174C15
:10FCE00034234B43E218D07892F802E0A0EB0E01E7
:10FCF000C9B2042902D1C120BDE8F08100F003019E
:10FD00000130C0B24FF00C0C0CFB0133D070A0EBF3
:10FD10000E001C44C0B2012825716671A760A4F8CA
:10FD20000C8007D143463A4631462846BDE8F041AB
:10FD300000F0BEB90020BDE8F08100BFC0FFFF1F8A
:10FD4000014B00201960704764000020024B0979C4
:10FD5000197100F08DBF00BF6400002013B50024AE
:10FD600002AA1C80044B42F8041D0979197100F0A5
:10FD70008DFF02B010BD00BF64000020002018807D
:10FD8000704730B40C460221198021796488084DEF
:10FD9000012C297102D130BC00F08EBF022C02D19F
:10FDA00030BC00F095BF0020188030BC704700BF09
:10FDB0006400002030B40C46022119802179648847
:10FDC000074D012C297102D130BC00F08DBF022CEF
:10FDD00002D130BC00F09ABF0020188030BC7047C0
:10FDE00064000020044B054A19795B791171137284
:10FDF00003210A23FFF75EBF640000205280FF1F2B
:10FE0000F8B500271F808B780B4CA371C3F3400318
:10FE10005A0063F3000206466271FFF7E3FF2568AC
:10FE200045B1A37913F002021ABF3A4622212121DB
:10FE30003046A8470020F8BD64000020034B00F1C5
:10FE400008021B6800780521184700BF6C000020DD
:10FE500070B5094D04462A1D012100F0D7FF80220C
:10FE60000121204600F0EAFF2B68207800220A21B9
:10FE7000BDE87040184700BF6C00002037B5012175
:10FE80000DF10702044600F0C1FF9DF80730074D51
:10FE9000802B04D12A790121204600F0CFFF2B6866
:10FEA000207800220B21984703B030BD6C00002061
:10FEB000436805215A7800F0C1BF73B501220024C0
:10FEC00005460126002100F089FF334621468DE8D2
:10FED00050001022284600F05FFF224621462846A7
:10FEE00000F07CFF234621468DE850001022284672
:10FEF00000F052FF31460222284600F09FFF3246B2
:10FF00000621284600F09AFF22469021284600F05C
:10FF100095FF044B28781B682246214602B0BDE8B5
:10FF2000704018476C00002042783AB9C178C90186
:10FF300041F0100101F0900100F080BF704773B5EF
:10FF40000C468DF8070001F00DFA1F4D2C60044699
:10FF5000002836D11D4A9DF80700102100F0A6FFA9
:10FF60001B4A044612219DF8070000F09FFF194A22
:10FF7000044314219DF8070000F098FFE4B2044305
:10FF8000154A9DF80700132100F090FFE4B20443E6
:10FF9000124A9DF80700172100F088FF02AEE4B274
:10FFA00004430F4A16F8010D162100F07FFFE4B25A
:10FFB000044303220121304600F040FF0323E4B252
:10FFC0002B71204602B070BD6C000020BBFE00000B
:10FFD000B1FE000051FE00007DFE000029FF000080
:10FFE0003DFE000037B502AD174B05F8010D0022AC
:10FFF000102128461A6000F05BFF122104462846B3
:020000021000EC
:1000000000F056FF14210443284600F051FFE4B2EB
:1000100004431321284600F04BFFE4B204431721A8
:10002000284600F045FFE4B204431621284600F0BC
:100030003FFFE4B2204310F0FF0003D19DF807001A
:1000400001F09CF903B030BD6C0000201FB5012108
:100050008DF807000DF10E020DF1070000F0D6FE3D
:100060000DF10F0206210DF1070000F0CFFE9DF803
:100070000E30802B18D19DF80F309B0714D59DF8BA
:10008000070000F0EFFD012804460DD172B60DF116
:10009000070000F029FB002221460DF107008DF832
:1000A0000E2000F0CBFE62B69DF80E0004B010BD2D
:1000B00073B50C4615461E468DF80700FFF7C6FFC0
:1000C000802808D033462A4621460DF1070000F06B
:1000D000A7FA02B070BD0020FBE77047062812D8CF
:1000E00080000129C0B201D10230C0B2074AC0F37A
:1000F0004703122101FB03231A884FF6FF739A422C
:1001000008BFFF207047FF20704700BF7400002029
:100110002DE9F041314C324D324E4FF0000884F859
:1001200000814FF4107285F840020F462846FF21E7
:1001300001F0D0FE4FF4806241463046C5F844627B
:1001400001F0C8FE94F80C3143F0800384F80C31C0
:1001500094F80C311B06FBD4234BFF221A7094F841
:100160000C3143F0400384F80C31204B196897B3ED
:1001700041F000411960194B310AC6F3074201F002
:10018000FE0183F89C1083F8B020320E83F8B4206F
:10019000174AC5F84822102283F80821012283F863
:1001A0009420BF2283F8802093F8002102F07F0280
:1001B00083F8002193F8842042F0010283F8842020
:1001C00093F8842042F0100283F8842084221A7766
:1001D0000020BDE8F08121F00041CBE7002007407E
:1001E00074000020000C00205C80FF1F00700440A1
:1001F000000E00200D4B93F80C2102F0BF0283F893
:100200000C21BF2283F8802093F8842002F0FE02A4
:1002100083F8842093F8942002F0FE0283F894205F
:100220001A7F02F07B021A770020704700200740F7
:10023000F7B5082304248DE81800B1F803300D78D1
:100240008878B3F5007F81BF0023CB7002230B7148
:10025000062D71D8AB00DCB2012804BF0234E4B231
:100260004FEA540E354C122707FB0E474FF6FF7628
:10027000B7F800C0B4455FD14E78032E5CD8012892
:100280005AD897F80FC0BCF1FF0F04BF4FF0000C15
:1002900087F80FC0B1F803C0122101FB0EFE04EB7A
:1002A0000E0743EA4003BA73FA7B7E7402F0010240
:1002B00013435BB2D4F84822C7F80220D9B2F973CD
:1002C0003874D4F8447224F80EC01BB207EBC30E86
:1002D00081F00101CEF80420AEF802C04FF0080E04
:1002E00007F833E007EBC10ECEF80420AEF802C0E9
:1002F00012FA8CF24FF0480E07F831E0C4F84822A9
:1003000028B917F8332062F07F0207F8332002AAD9
:1003100002EB80002DB20A4950F8082C11F8253064
:10032000012E0CBF164642F001063343DBB201F842
:100330002530002003B0F0BD9520FBE774000020BD
:10034000C0200740084610B51146FFF7C7FEFF283A
:100350001DD0104B1221C0F3470001FB0030D3F831
:100360004422C37B1CB283F0010312F8341001F065
:100370007F0102F8341012F8331001F07F0102F807
:1003800033104FF0FF338372C372002010BDC420BE
:1003900010BD00BF7400002073B50C468DF8070037
:1003A000114620461646FFF799FEFF28054620D045
:1003B000214632460DF10700FFF7C4FFC5F347039E
:1003C00012210D4D59436B18D5F848221888121A7E
:1003D000C5F8482224B2094A002002F824004FF050
:1003E000FF326A549A705A70DA701A715A7102B0F8
:1003F00070BD9620FBE700BF74000020C0200740BE
:100400002DE9F0410E468046114630461746FFF76B
:1004100065FE0C4DC0F34700122303FB0050C47B64
:10042000FF2C0DD03A4631464046FFF78BFF24B2F1
:10043000D5F8442212F8343063F07B0302F83430EC
:10044000BDE8F0817400002010B508460021144674
:10045000FFF744FE084AC0F34700122101FB0020C9
:10046000D2F84432C27B03EBC2035A68136823609C
:100470005368636010BD00BF7400002010B50C46C7
:1004800020461146FFF72AFEFF281AD024B2104B4F
:1004900013F82430DBB213F00C0F12D09B0712D4E8
:1004A0000C4BD3F8443213F83020D2090DD180F030
:1004B0000100C0B213F83030DB0914BF0320002064
:1004C00010BD052010BD012010BD032010BD00BFD0
:1004D000C02007407400002008B5FFF7FFFD074A61
:1004E0001223C0F3470003FB0020C37BFF2B1EBF7A
:1004F000D2F84422002102F8331008BD7400002015
:100500002DE9F0410846002190461F46FFF7E6FD21
:100510002249C0F34700122404FB0014E57BFF2DA1
:1005200039D022884FF6FF7093B2834233D0D1F88E
:10053000441285F0010011F9300000282BDB2EB2A7
:1005400087B901EBC60338465A80D4F802205A60B6
:1005500011F8352002F0400262F0770201F83620EF
:10056000BDE8F08101EBC602BB424FF0000028BF9E
:100570003B466781C4F80680207360735380C2F8DD
:10058000048011F8353003F0400363F0770301F87D
:100590003630BDE8F0819420BDE8F0817400002081
:1005A0002DE9F0410C460646114620461546FFF758
:1005B00095FD194BC0F34700122202FB003090F862
:1005C0000FE0BEF1FF0F24D027B2144A6CB1407C7B
:1005D000012D0CBF14211821012818BF41F0010181
:1005E00012F82700014302F8271012F827106FF3C2
:1005F000410102F82710D3F84432002203F83E20CC
:100600003DB92B462A4621463046BDE8F041FFF76A
:1006100077BFBDE8F08100BF74000020C020074014
:100620002DE9F0410C462046012117469846FFF778
:1006300055FDFF2836D01C4BC0F34700122202FBA9
:100640000030D3F8446290F80FE016F93E30002BEA
:1006500028DB23B2154A12F8235015F0020521D1E8
:100660000188C0F806701FFA88F242818A42D8BF1A
:1006700011460FFA8EF206EBC203057345735980DB
:100680005F602CB9C82306F832302046BDE8F081FF
:1006900016F83E3003F0400363F0770306F832307B
:1006A0002C46F2E79324F0E774000020C0200740B6
:1006B000034B044883F898100122114600F0BEBB9A
:1006C00000200740B4020020054B0648002283F8B2
:1006D0009420802283F80C210121FF2200F0AEBB80
:1006E00000200740B402002038B51A4C94F80021CD
:1006F00002F07F0284F8002194F80C2102F0DF025E
:1007000084F80C2194F8802042F0200284F88020A4
:1007100094F8842002F0DF0284F8842094F8942076
:1007200002F0DF0284F8942094F8942042F004024E
:1007300084F8942044F62065013DADB200F0BCFE83
:10074000002DF9D194F8943003F0FB0384F8943031
:1007500038BD00BF002007402DE9F04FD84DD94CDF
:1007600095F8807095F8843095F8906087B0FF22F6
:100770001F4094F840328DF809208DF80C308DF828
:100780000D20002301210DF1090204F510708DF8F0
:100790000E3004938DF815308DF816308DF80F302B
:1007A0008DF8143000F032FB95F80C31D907F6B211
:1007B0000FD59DF80930802B0BD195F8003103F04F
:1007C0007F0385F8003195F80C3103F0DF0385F8DD
:1007D0000C317A0711D5BA4B042093F8A41093F882
:1007E000A02083F8800006AB42EA012223F80E2DF8
:1007F00003A91220049300F06DFBFB074BD5B04D0D
:10080000B0480123BF2685F8803085F8886095F8C8
:100810009430002743F0020385F894304FF41072AF
:1008200085F89870FF2185F8007101F053FB4FF4B3
:1008300080623946D4F8440201F04CFBD4F84432CB
:1008400003F50073C4F848329F4BFF221A7095F8E5
:10085000943003F0FD0385F8943095F80C3143F0A3
:10086000400385F80C319F2385F88C6085F884302F
:1008700095F8943003F0DF0385F8943003A9102035
:1008800000F028FB95F8943003F0DF0385F89430EE
:1008900007B0BDE8F08F3D0740F19380884B0822F8
:1008A00083F880203309C6F3C000062B8DF80D3085
:1008B0008DF80F0000F2F480C6F3800202EB830291
:1008C00008B10232D2B2D4F8446206EBC201C2F3DC
:1008D0004705D1F804E04988ADF81510122101FB55
:1008E0000541CDF810E091F80FC08CF0010C81F8B3
:1008F0000FC016F8321082F0010A5FFA8AFAC1F3CB
:1009000080110FFA8AF881F00101890106EBC8090C
:1009100006F83810002800F0D980DFF8ACB19BB998
:100920009BF8002082B9FF2219468BF8002003A80B
:100930001A460193FFF706FD019B06F838301A4668
:10094000194603A8FFF7DCFD9BF80030012B04D00B
:100950009DF80D30002B00F0AD80122101FB054108
:10096000BDF815008B894A8903449BB293428B8161
:1009700009D3B1F800E0C0B2864540F09380897B8E
:10098000012940F08F80122101FB0544D4F80610A4
:1009900020881944D31A8342D8BF98B2A9F802001C
:1009A000C9F8041016F83A3003F0400363F07703F7
:1009B00006F83830424A92F8943003F0DF0382F8A8
:1009C0009430B80717D53E4C022384F8803094F851
:1009D000883094F88C2003A9134016208DF8143029
:1009E00000F078FABF2384F8883094F8943003F04C
:1009F000DF0384F89430F9061CD5314C202384F8A9
:100A00008030102384F8803003A9142000F062FAAB
:100A100094F80C3143F0200384F80C3194F8003141
:100A200043F0800384F8003194F8843043F02003CD
:100A300084F88430BA060DD5214C202384F8803008
:100A400003A9132000F046FA94F8843003F0DF0382
:100A500084F884303B067FF51BAF0DF10A02FF23BB
:100A6000102103A88DF80D3000F0D0F99DF80A3060
:100A7000134C012B04BF8DF80F3000224FF0800380
:100A800008BF8DF80D2003A984F88030172000F0EE
:100A900021FA94F8943003F0DF0384F89430F7E6F9
:100AA000FF2210E7122202FB0544D4F8062004922C
:100AB000ADF8153003A99DF80D0000F00BFA79E7A9
:100AC00000200740740000205C80FF1F6BB916F8FF
:100AD00032202F4902F03C02342A35D101238DF80F
:100AE0000E309EF80030DB090B70122101FB05412E
:100AF0004FF6FF734A899A42DCD0BDF815E08B8926
:100B000073449BB28B8109888E4501D19A420CD8DF
:100B10008AB3B2FBF1F001FB102080B258BB122067
:100B200000FB0540807B012825D1D21A8A42D8BF1C
:100B300091B2122202FB0544C9B9D4F80230C9F8B7
:100B40000430A9F802102DE70A78012ACDD1FF2040
:100B50000870194603A80193FFF7F4FB019B06F800
:100B600038301A46194603A8FFF7CAFCBDE7D4F887
:100B700006201344E3E7122202FB0544D4F80620C2
:100B8000ADF815304FF0FF330492A372E37291E792
:100B90005C80FF1F13460A46194601F09BB900BF4F
:100BA00030B50329039C04981DD12BB9164A226045
:100BB00004220280002030BD40F209418B420FD157
:100BC000022A4FF000030CD810490C2505FB031333
:100BD000D9681B6951F8221021609B5C0380E9E70A
:100BE00001230122F0E7072901D9CD2030BD074BB1
:100BF00003EB8102126A2260002AF6D003EB410364
:100C0000B3F84030EAE700BF5D80FF1F0422010017
:100C100001299FBF034B5B5C1370002088BFCD2070
:100C2000704700BFC002002001299DBF024B002079
:100C30005A54CD20704700BFC002002019B14B1E8E
:100C400058425841704701207047054B1A788A4234
:100C500004D05878431A58425841704701207047D1
:100C6000C002002000207047004870475422010055
:100C700001299FBF044BC1EBC101C918002094BFDB
:100C80001160CD20704700BF6180FF1F012930B582
:100C90000ED8084DC1EBC10108231068C45CC81808
:100CA000284401330F2B00F8084CF6D1002030BD4A
:100CB000CD2030BD6180FF1F01299FBF034B03EB97
:100CC00041010020116088BFCD207047C202002082
:100CD00001299FBF034B03EB41010020116088BF36
:100CE000CD207047C602002001290AD81368187861
:100CF000054B03EB4101887013685B78CB700020D3
:100D00007047CD20704700BFC002002001290AD8DB
:100D100013681878054B03EB4101887113685B7801
:100D2000CB7100207047CD20704700BFC00200206B
:100D3000084B5A7803F8022BFF210022D1540132CC
:100D4000072AFBD1044A0023052199540133072BBC
:100D5000FBD17047CA020020D302002000BF7047B9
:100D6000013AD2B2062A10B51C4608D8054B5A7073
:100D7000FFF7DEFF2146BDE81040FFF7C9B9992013
:100D800010BD00BFCA020020024B00225A70FFF7BC
:100D900031BA00BFCA02002037B50F4C257805B91B
:100DA000C1B98DF802308DF800109DF81830ADF8FB
:100DB000032069469DF81C2000788DF80130FFF76C
:100DC00037FA9DF800301BB110B92378013B23702E
:100DD00003B030BD9520FBE7CA02002038B50A4BAE
:100DE0000D461C7859788C421C4600D14DB92946D5
:100DF0000078FFF7D1FA2DB120B9237801332370A1
:100E000038BD962038BD00BFCA0200204B1E062BFD
:100E100005D8094B19444B78137000207047CB0656
:100E200007D501F00F01062903D8034B19444B7A6B
:100E3000F2E78220704700BFCA0200204B1E062B3B
:100E40002DE9F0418046174605D8174B19444A70E2
:100E50000020BDE8F081CB0622D501F00F05062D5C
:100E60001ED8012A4FEAD1140F4E06D12246294638
:100E7000FFF7C6FA35446F72EAE7002AFAD1731910
:100E80005B7A012BF6D122462946FFF789FB002D1C
:100E9000F0D184F0010229464046FFF781FBE9E7E3
:100EA0008220BDE8F08100BFCA0200200020704708
:100EB000062903D9A1F11003072B07D8044B53F8D7
:100EC0002130002B0CBFC42000207047C420704785
:100ED0007C220100102810B50C4601D1FFF728FF35
:100EE000034B53F820300BB120469847002010BD2B
:100EF0007C2201001FB5144602228DF807001A80DB
:100F000005210DF10F020DF10700FFF77FFF034BE5
:100F10009DF80F201A80236004B010BDDC02002071
:100F20001FB5144601228DF807001A8004210DF127
:100F30000F020DF10700FFF769FF044B9DF80F202A
:100F40001A800020236004B010BD00BFDC02002026
:100F5000F0B5002685B01E8049888DF80700ADF8F1
:100F60000E10FFF76BFE18B3BDF80E20114F04AC46
:100F7000B2FA82F2520901210DF10700FFF75EFF7C
:100F800034F8022D0421D2B20DF10700FFF756FF0D
:100F90007B682246012105469DF8070098477B683B
:100FA0009DF80700324602219847284605B0F0BD5B
:100FB0000425FAE7DC02002073B502AC002504F832
:100FC000010D0E461D80042201212046FFF736FF49
:100FD0007288024B28461A7202B070BDDC020020F3
:100FE00013B54C8889888DE80C000B46E2B2210AC3
:100FF000FFF7D6FD02B010BD2DE9F04186B01746CF
:101000001E4606AA00238846059303238DF80F0089
:1010100002F8083D01210DF10F00FFF7F7FE98F8E7
:101020000050274C15F0030528D10DF111020621BF
:101030000DF10F00FFF7EAFE9DF811309DF80F004B
:1010400003F0030323800DF11203019305AB00931A
:101050002A462B460221FFF7A3FD059BDB7913F0FF
:10106000400F238814BF43F0010323F001032380C2
:10107000022333803C6006B0BDE8F081012D08D129
:101080009DF81030012B02D198F80430ABB9002341
:10109000EDE7022DEED198F8041041F010010DF1AA
:1010A0001202C9B20DF10F00FFF7B0FE9DF8123029
:1010B00003F0010323803580DCE7CD20DAE700BFB1
:1010C000DC0200207FB500221A800B784E788DF864
:1010D000070013F003030D46C6F3400634D1FEB1FA
:1010E0004B88013B9BB2012B52D80DF10F02062118
:1010F0000DF10700FFF78AFE044670B9AB780122B4
:101100009A409DF80F301A43D2B206210DF1070024
:101110008DF80F20FFF792FE0446204604B070BD04
:101120004E88012E34D10DF10F0206210DF107007A
:10113000FFF76CFE04460028EFD1AA7896409DF890
:101140000F2022EA0602E0E7022B21D109798DF86F
:101150000F10324641F010010DF10700FFF76EFE4F
:101160006B78002E14BF07210821012B044607D1FC
:101170009DF80F00C10900F00F00FFF7ADF908213D
:10118000044B9DF807005B680DF10F029847C4E718
:10119000CD24C2E7DC02002010B500241C800B78AF
:1011A00003F00303012B05D18A780979FFF73CFD91
:1011B000204610BD042010BD38B515460A7802F04F
:1011C0000302012A07D1054C1A8009792246FFF74C
:1011D0001FFD2C6038BD042038BD00BFDC0200209C
:1011E00013B5CD298DF8070007D1012290210DF10B
:1011F0000700FFF723FE02B010BD0D491C88088AC6
:101200001268844288BF18800C461B889DF807002E
:101210000021FEF74DFF94F90A30002BEBDA002392
:101220001A4619460DF10700FFF76AF9E3E700BF18
:10123000DC02002073B5054600266A4601218DF8C0
:1012400000600196FFF7E2FDAA78434C012A52D1D3
:1012500068680368C4F80A304368A07AC4F80E309E
:1012600004F10A0110F0600F1ED1E27A3B4B53F8F3
:101270002240002C3DD09DF80000022839D802EB16
:1012800042021344034493F83430012B31D10DF161
:10129000020301AA2878A0470DF1020301AA014622
:1012A0002878FFF79DFF13E0238AADF80230202B4A
:1012B00017D87BB102060DD40A68C4F812204A6818
:1012C000C4F81620314604F11A022846FFF718F92F
:1012D00002B070BDE46B64B10DF1020301AA2049B4
:1012E000D8E702A82B7800F8073D9021FFF7A6FD6C
:1012F000EEE7CD20D0E79DF80030042B10D12B78FD
:10130000217A02AD05F8063D2846FFF7D1F9012202
:1013100011462846FFF792FD227A03212846E5E789
:1013200094F90A30002BD3DBEB78002BD0D1E66B9D
:1013300086B1B5F8093028780833ADF8023004F1E9
:1013400012010DF1020301AAB04701460DF102039B
:1013500001AAA5E7CD21F9E7DC020020DC2201008B
:10136000E6020020034B5960DA630021024AFFF7CE
:101370009DBD00BFDC0200203512010007B502ABA5
:10138000054A03F8010D002118465160D163FFF7AB
:101390008FFD03B05DF804FBDC02002000207047E5
:1013A000354B41F248015A5822F00F0242F0020236
:1013B0005A5041F204015A5842F480225A5041F2E4
:1013C00034015A5842F480225A5003F52C336021DC
:1013D00093F8942042F0020283F89420C02283F80C
:1013E0000021FF221A7483F8802083F8882083F874
:1013F0008420002283F88C2083F80C111F491A7571
:10140000080A00F0FE0083F8982083F8C02083F8D3
:10141000C42083F8C82083F8CC2083F8D02083F838
:10142000D42083F8D82083F8DC2083F8E02083F8E8
:10143000E42083F8E82083F8EC2083F8F02083F898
:10144000F42083F8F82083F8FC2083F89C00C1F393
:101450000740090E83F8B00083F8B41083F8AC207D
:101460001A7783F8082193F8942002F0D40242F00E
:10147000010283F89420704700700440000C0020A3
:10148000024B4FF400125A60704700BF00E100E0C9
:10149000034B4FF40012C3F884215A60704700BF19
:1014A00000E100E008B5FEF782F910B9FFF7F0FFA0
:1014B00008BD1B2008BD00BF034B4AF202629A819F
:1014C0004BF280429A81704700200540844641EAF1
:1014D000000313F003036DD1403A41D351F8043BAC
:1014E00040F8043B51F8043B40F8043B51F8043BFE
:1014F00040F8043B51F8043B40F8043B51F8043BEE
:1015000040F8043B51F8043B40F8043B51F8043BDD
:1015100040F8043B51F8043B40F8043B51F8043BCD
:1015200040F8043B51F8043B40F8043B51F8043BBD
:1015300040F8043B51F8043B40F8043B51F8043BAD
:1015400040F8043B51F8043B40F8043B51F8043B9D
:1015500040F8043B51F8043B40F8043B403ABDD20C
:10156000303211D351F8043B40F8043B51F8043BAE
:1015700040F8043B51F8043B40F8043B51F8043B6D
:1015800040F8043B103AEDD20C3205D351F8043B3D
:1015900040F8043B043AF9D2043208D0D2071CBF09
:1015A00011F8013B00F8013B01D30B880380604632
:1015B000704700BF082A13D38B078DD010F00303A8
:1015C0008AD0C3F10403D21ADB071CBF11F8013B18
:1015D00000F8013B80D331F8023B20F8023B7BE767
:1015E000043AD9D3013A11F8013B00F8013BF9D292
:1015F0000B7803704B7843708B788370604670472C
:1016000081F0004102E000BF83F0004330B54FEAB3
:1016100041044FEA430594EA050F08BF90EA020F20
:101620001FBF54EA000C55EA020C7FEA645C7FEAB3
:10163000655C00F0E2804FEA5454D4EB5555B8BFD6
:101640006D420CDD2C4480EA020281EA030382EA47
:10165000000083EA010180EA020281EA0303362DD9
:1016600088BF30BD11F0004F4FEA01314FF4801CAC
:101670004CEA113102D0404261EB410113F0004FBE
:101680004FEA03334CEA133302D0524263EB430375
:1016900094EA050F00F0A780A4F10104D5F1200E13
:1016A0000DDB02FA0EFC22FA05F2801841F100016E
:1016B00003FA0EF2801843FA05F359410EE0A5F142
:1016C00020050EF1200E012A03FA0EFC28BF4CF073
:1016D000020C43FA05F3C01851EBE37101F0004529
:1016E00007D54FF0000EDCF1000C7EEB00006EEB36
:1016F0000101B1F5801F1BD3B1F5001F0CD34908C0
:101700005FEA30004FEA3C0C04F101044FEA445216
:1017100012F5800F80F09A80BCF1004F08BF5FEA9D
:10172000500C50F1000041EB045141EA050130BD7D
:101730005FEA4C0C404141EB010111F4801FA4F120
:101740000104E9D191F0000F04BF01460020B1FA75
:1017500081F308BF2033A3F10B03B3F120020CDAAD
:101760000C3208DD02F1140CC2F10C0201FA0CF08B
:1017700021FA02F10CE002F11402D8BFC2F1200CF0
:1017800001FA02F120FA0CFCDCBF41EA0C019040A6
:10179000E41AA2BF01EB0451294330BD6FEA0404EF
:1017A0001F3C1CDA0C340EDC04F11404C4F12002DA
:1017B00020FA04F001FA02F340EA030021FA04F3EC
:1017C00045EA030130BDC4F10C04C4F1200220FA43
:1017D00002F001FA04F340EA0300294630BD21FA81
:1017E00004F0294630BD94F0000F83F4801306BF47
:1017F00081F480110134013D4EE77FEA645C18BF3B
:101800007FEA655C29D094EA050F08BF90EA020FD1
:1018100005D054EA000C04BF1946104630BD91EAC9
:10182000030F1EBF0021002030BD5FEA545C05D1CC
:101830004000494128BF41F0004130BD14F580040B
:101840003CBF01F5801130BD01F0004545F0FE417F
:1018500041F470014FF0000030BD7FEA645C1ABFB4
:10186000194610467FEA655C1CBF0B46024650EAEB
:10187000013406BF52EA033591EA030F41F4002117
:1018800030BD00BF90F0000F04BF0021704730B59D
:101890004FF4806404F132044FF000054FF0000172
:1018A00050E700BF90F0000F04BF0021704730B533
:1018B0004FF4806404F1320410F0004548BF404208
:1018C0004FF000013EE700BF42004FEAE2014FEA5D
:1018D00031014FEA02701FBF12F07F4393F07F4F38
:1018E00081F06051704792F0000F14BF93F07F4F6A
:1018F000704730B54FF4607401F0004521F00041AD
:1019000020E700BF50EA010208BF704730B54FF032
:1019100000050AE050EA010208BF704730B511F037
:10192000004502D5404261EB41014FF4806404F16F
:1019300032045FEA915C3FF4DCAE4FF003025FEAF1
:10194000DC0C18BF03325FEADC0C18BF033202EB79
:10195000DC02C2F1200300FA03FC20FA02F001FAD3
:1019600003FE40EA0E0021FA02F11444C1E600BF72
:1019700070B54FF0FF0C4CF4E06C1CEA11541DBF25
:101980001CEA135594EA0C0F95EA0C0F00F0DEF8F0
:101990002C4481EA030621EA4C5123EA4C5350EAD5
:1019A000013518BF52EA033541F4801143F4801326
:1019B00038D0A0FB02CE4FF00005E1FB02E506F0B7
:1019C0000042E0FB03E54FF00006E1FB03569CF00C
:1019D000000F18BF4EF0010EA4F1FF04B6F5007F12
:1019E00064F5407404D25FEA4E0E6D4146EB060684
:1019F00042EAC62141EA55514FEAC52040EA5E500D
:101A00004FEACE2EB4F1FD0C88BFBCF5E06F1ED8B6
:101A1000BEF1004F08BF5FEA500E50F1000041EBED
:101A2000045170BD06F0004646EA010140EA02009A
:101A300081EA0301B4EB5C04C2BFD4EB0C0541EABC
:101A4000045170BD41F480114FF0000E013C00F3D1
:101A5000AB8014F1360FDEBF002001F0004170BDF5
:101A6000C4F10004203C35DA0C341BDC04F114040E
:101A7000C4F1200500FA05F320FA04F001FA05F29A
:101A800040EA020001F0004221F0004110EBD37067
:101A900021FA04F642EB06015EEA430E08BF20EA93
:101AA000D37070BDC4F10C04C4F1200500FA04F336
:101AB00020FA05F001FA04F240EA020001F00041C8
:101AC00010EBD37041F100015EEA430E08BF20EA3B
:101AD000D37070BDC4F1200500FA05F24EEA020E83
:101AE00020FA04F301FA05F243EA020321FA04F0B2
:101AF00001F0004121FA04F220EA020000EBD37069
:101B00005EEA430E08BF20EAD37070BD94F0000F68
:101B10000FD101F00046400041EB010111F4801F9C
:101B200008BF013CF7D041EA060195F0000F18BF4D
:101B3000704703F00046520043EB030313F4801F89
:101B400008BF013DF7D043EA0603704794EA0C0F43
:101B50000CEA135518BF95EA0C0F0CD050EA410659
:101B600018BF52EA4306D1D181EA030101F00041D6
:101B70004FF0000070BD50EA410606BF10461946FE
:101B800052EA430619D094EA0C0F02D150EA01360A
:101B900013D195EA0C0F05D152EA03361CBF10464B
:101BA00019460AD181EA030101F0004141F0FE41EA
:101BB00041F470014FF0000070BD41F0FE4141F46E
:101BC000780170BD70B54FF0FF0C4CF4E06C1CEA6E
:101BD00011541DBF1CEA135594EA0C0F95EA0C0F23
:101BE00000F0A7F8A4EB050481EA030E52EA0335DE
:101BF0004FEA013100F088804FEA03334FF08055FF
:101C000045EA131343EA12634FEA022245EA11152B
:101C100045EA10654FEA00260EF000419D4208BFDC
:101C2000964244F1FD0404F5407402D25B084FEA89
:101C30003202B61A65EB03055B084FEA32024FF435
:101C400080104FF4002CB6EB020E75EB030E22BF92
:101C5000B61A754640EA0C005B084FEA3202B6EB52
:101C6000020E75EB030E22BFB61A754640EA5C0001
:101C70005B084FEA3202B6EB020E75EB030E22BF91
:101C8000B61A754640EA9C005B084FEA3202B6EB92
:101C9000020E75EB030E22BFB61A754640EADC0051
:101CA00055EA060E18D04FEA051545EA16754FEAB3
:101CB00006164FEAC30343EA52734FEAC2025FEAD1
:101CC0001C1CC0D111F4801F0BD141EA00014FF060
:101CD00000004FF0004CB6E711F4801F04BF014331
:101CE0000020B4F1FD0C88BFBCF5E06F3FF6AFAE4D
:101CF000B5EB030C04BFB6EB020C5FEA500C50F1DD
:101D0000000041EB045170BD0EF0004E4EEA11315F
:101D100014EB5C04C2BFD4EB0C0541EA045170BD66
:101D200041F480114FF0000E013C90E645EA060EAA
:101D30008DE60CEA135594EA0C0F08BF95EA0C0FD8
:101D40003FF43BAF94EA0C0F0AD150EA01347FF420
:101D500034AF95EA0C0F7FF425AF104619462CE7F7
:101D600095EA0C0F06D152EA03353FF4FDAE10465A
:101D7000194622E750EA410618BF52EA43067FF4AB
:101D8000C5AE50EA41047FF40DAF52EA43057FF43B
:101D9000EBAE12E74FEA410212F5001215D211D54F
:101DA0006FF47873B3EB625212D94FEAC12343F058
:101DB000004343EA505311F0004F23FA02F018BFDA
:101DC000404270474FF00000704750EA013005D1A3
:101DD00011F0004008BF6FF0004070474FF0000066
:101DE000704700BFFDF7ABFB002103E00A4B5B58D7
:101DF0004350043109480A4B42189A42F6D3094A23
:101E000002E0002313600432074B9A42F9D300F03A
:101E10000DF8804770470000682301000880FF1F0D
:101E20007485FF1F0086FF1F24100020264C08B574
:101E3000F6F727FBF6F78EFBF6F7F4FCF6F706FD50
:101E4000F6F710FCF6F7F2FEFCF73EFCFCF726FA7C
:101E5000F7F783F8F6F79CFD2078F6F713FCE078A7
:101E6000F6F780FCF6F73DFE28B1F6F73AFE607013
:101E7000F6F737FEA060F6F7B5FE21896079228A71
:101E8000FCF766FAFDF752FAFDF7DFF8FCF7B2FC53
:101E90000E4B4FF400725A60F8F73CF8FBF750F81D
:101EA0000B4B04229A60FAF7A7FCFBF72DF9FBF71E
:101EB00048F8F6F74AFEF6F785FE0028F3D0FDF75E
:101EC000C4F8F8F727F8EEE70C80FF1F80F00F400A
:101ED00000F00F4070B4860746D0541E002A41D04F
:101EE000CAB2034602E014F1FF343BD303F8012BDE
:101EF0009D07F8D1032C2ED9CDB245EA05250F2C2C
:101F000045EA054519D903F110022646103E0F2E69
:101F100042F8105C42F80C5C42F8085C42F8045C41
:101F200002F11002F2D8A4F1100222F00F0204F024
:101F30000F041032032C13440DD91E462246043AD6
:101F4000032A46F8045BFAD8221F22F00302043267
:101F5000134404F003042CB1C9B21C4403F8011B60
:101F60009C42FBD170BC704714460346C2E700BFD9
:101F7000024B13B1024800F005B8704700000000A2
:101F8000911F0100002301461A46184600F01EB8B2
:101F900038B50A4C0A4D641BA4100AD004F18043E2
:101FA000013B05EB8305013C55F804399847002CAB
:101FB000F9D1BDE8384000F0CBB900BF682301007B
:101FC00064230100704700BF704700BF2DE9F8434C
:101FD0002C4D0646286898460F469146FFF7F2FFBB
:101FE000294B1C68D4F84831002B3ED05A681F2A70
:101FF0001CDC02F1010E76B103EB82010124C1F871
:102000008890D3F8880194402043022EC3F88801B9
:10201000C1F8088123D00232C3F804E0286843F8ED
:102020002270FFF7D1FF0020BDE8F883174B0BB3F8
:102030004FF4C870AFF300800346D8B1D4F84821FC
:102040000260002141600A46C4F848014FF0010EC9
:10205000C0F88811C0F88C11002EDCD0CCE7D3F882
:102060008C110C43C3F88C41D5E704F5A673C4F872
:102070004831BBE72868FFF7A7FF4FF0FF30BDE806
:10208000F88300BF7085FF1F40230100000000009F
:102090008025000040380000004B000080700000E8
:1020A0000096000000E10000002C010000C20100C9
:1020B0000084030090D0030020A1070040420F00DD
:1020C00000000000E0930400C0270900FF00FF00AB
:1020D0000000000064F00000E8030000102700008A
:1020E00010270000140000000A000000000000009B
:1020F000FFFFFF3F000001006400000064000000DB
:1021000000070000F40100000000000000000000D3
:1021100000000000000000000000000000000000BF
:102120000050C300008813000140080800000000B0
:1021300000000000C8000000010000000080000056
:1021400000000000000000000000C80000200300A4
:10215000000000000000000000000000C8000000B7
:10216000000000000000000000000000000000006F
:10217000000000000000000000000000000000005F
:10218000000000000001010001000000010000004B
:10219000010000000000010000000000000000003D
:1021A000000000000101010000000000000000002C
:1021B0000001000000000000010101000101000118
:1021C000010000000000000000000000000000000E
:1021D00000000000000000000000000000000000FF
:1021E00000000000000000000000000000000101ED
:1021F00000000001000101010000000000000000DB
:10220000000000005D80FF1F0400000009040000C2
:102210006822010078220100000000000000000098
:1022200000000000000000003481FF1FF180FF1F4C
:10223000000000000000000000000000000000009E
:102240000000000000001200430000000000000039
:102250000000000003010201100002020010000350
:1022600003011000000100005D80FF1FB780FF1F09
:102270009180FF1F6F80FF1F043A26223512010054
:1022800031FB0000C9FB000039F900005D0D0100C1
:102290005D0D01005D0D01005D0D01005D0D010092
:1022A0005D0D01005D0D01005D0D01005D0D010082
:1022B0005D0D01005D0D01005D0D0100BBFE000024
:1022C00051FE0000B1FE00007DFE000051FE000046
:1022D0005D0D01003DFE000029FF0000F90F010027
:1022E000C510010000000000C51001000000000042
:1022F000B90F0100E10F010000000000210F0100F3
:10230000510F0100B911010099110100F50E0100F2
:1023100001010001010000000001010000000000B7
:1023200001010101010000000101000101000100A3
:1023300000010000010000333331345631303900E0
:102340004881FF1FF8B500BFF8BC08BC9E46704727
:0C235000F8B500BFF8BC08BC9E46704702
:08235C00711F0100358400002F
:0423640011840000E0
:1023680037230100000102000008000001000000FE
:102378000200000000000000000000000000000053
:102388000000000000000000000000000000000045
:102398000000000000000000000000000000000035
:1023A80000000000010002000400A120000000005D
:1023B80002000000FF0403090400C2010000000835
:1023C80000000000000000220342004100440020F9
:1023D8000053005400520049004E004700200049B5
:1023E800004E004400450058002603530074006561
:1023F80000700070006500720020004D006F0074CE
:10240800006F007200200044006500760020003A4A
:10241800035400520049004E0041004D004900435A
:102428000020004D006F00740069006F006E0020EE
:102438000043006F006E00740072006F006C002093
:1024480000200020002000200009024300020100B3
:10245800C032090400000102020000052400100136
:1024680005240101010424020605240600010705CC
:10247800830310000A09040100020A00000007058E
:10248800810210000007050202100000120100027C
:10249800020000103C2A00010200010200010000B5
:1024A800000000003484FF1F9C84FF1F0485FF1F69
:1024B8000000000000000000000000000000000014
:1024C8000000000000000000000000000000000004
:1024D80000000000000000000000000000000000F4
:1024E80000000000000000000000000000000000E4
:1024F80000000000000000000000000000000000D4
:1025080000000000000000000000000000000000C3
:1025180000000000000000000000000000000000B3
:1025280000000000000000000000000000000000A3
:102538000000000000000000000000000000000093
:102548000000000000000000010000000000000082
:102558000E33CDAB34126DE6ECDE05000B00000047
:102568000000000000000000000000000000000063
:102578000000000000000000000000000000000053
:102588000000000000000000000000000000000043
:102598000000000000000000000000000000000033
:0C28C800000000000000000000100020D4
:1028D400682301000880FF1F6C0500000000000051
:0828E4000000000000000000EC
:020000020000FC
:020000041FFFDC
:04800000000000007C
:0400000310001DE5E7
:00000001FF
